 lua

 Timestamp is 54e2a59f (Mon Feb 16 20:21:19 2015)

 Preferred load address is 10000000

 Start         Length     Name                   Class
 0001:00000000 0000db6cH .text                   CODE
 0001:0000db6c 0000000aH .text$x                 CODE
 0001:0000db76 0000005eH .text$yc                CODE
 0001:0000dbd4 0000002cH .text$yd                CODE
 0002:00000000 000001e0H .idata$5                DATA
 0002:000001e0 00000004H .CRT$XCA                DATA
 0002:000001e4 00000018H .CRT$XCU                DATA
 0002:000001fc 00000004H .CRT$XCZ                DATA
 0002:00000200 00000004H .CRT$XIA                DATA
 0002:00000204 00000004H .CRT$XIAA               DATA
 0002:00000208 00000008H .CRT$XIC                DATA
 0002:00000210 00000004H .CRT$XIZ                DATA
 0002:00000220 00002168H .rdata                  DATA
 0002:00002388 00000068H .rdata$debug            DATA
 0002:000023f0 0000017cH .rdata$r                DATA
 0002:00002570 00000008H .rdata$sxdata           DATA
 0002:00002578 00000004H .rtc$IAA                DATA
 0002:0000257c 00000004H .rtc$IZZ                DATA
 0002:00002580 00000004H .rtc$TAA                DATA
 0002:00002584 00000004H .rtc$TZZ                DATA
 0002:00002588 00000134H .xdata$x                DATA
 0002:000026bc 00000064H .idata$2                DATA
 0002:00002720 00000014H .idata$3                DATA
 0002:00002734 000001e0H .idata$4                DATA
 0002:00002914 000006acH .idata$6                DATA
 0002:00002fc0 00000a08H .edata                  DATA
 0003:00000000 000000ecH .data                   DATA
 0003:00000100 00000794H .bss                    DATA
 0004:00000000 00000058H .rsrc$01                DATA
 0004:00000060 00000180H .rsrc$02                DATA

  Address         Publics by Value              Rva+Base       Lib:Object

 0000:00000000       __except_list              00000000     <absolute>
 0000:00000002       ___safe_se_handler_count   00000002     <absolute>
 0000:00009876       __fltused                  00009876     <absolute>
 0000:00009876       __ldused                   00009876     <absolute>
 0000:00000000       ___ImageBase               10000000     <linker-defined>
 0001:00000000       ??0_Ignore@std@@QAE@XZ     10001000 f i pch.obj
 0001:00000003       _luaA_index@8              10001003 f   lapi.obj
 0001:00000051       _luaA_pushobject@8         10001051 f   lapi.obj
 0001:0000007a       _lua_concat@8              1000107a f   lapi.obj
 0001:000000a5       _lua_equal@12              100010a5 f   lapi.obj
 0001:000000d9       _lua_getgccount@4          100010d9 f   lapi.obj
 0001:000000e6       _lua_getgcthreshold@4      100010e6 f   lapi.obj
 0001:000000f3       _lua_getglobal@8           100010f3 f   lapi.obj
 0001:00000132       _lua_getglobals@4          10001132 f   lapi.obj
 0001:0000015d       _lua_getn@8                1000115d f   lapi.obj
 0001:000001c3       _lua_getref@8              100011c3 f   lapi.obj
 0001:00000222       _lua_gettable@8            10001222 f   lapi.obj
 0001:00000260       _lua_gettop@4              10001260 f   lapi.obj
 0001:0000026f       _lua_insert@8              1000126f f   lapi.obj
 0001:000002a9       _lua_iscfunction@8         100012a9 f   lapi.obj
 0001:000002d0       _lua_isnumber@8            100012d0 f   lapi.obj
 0001:00000301       _lua_isstring@8            10001301 f   lapi.obj
 0001:00000322       _lua_lessthan@12           10001322 f   lapi.obj
 0001:00000359       _lua_newtable@4            10001359 f   lapi.obj
 0001:00000389       _lua_newuserdata@8         10001389 f   lapi.obj
 0001:000003c1       _lua_next@8                100013c1 f   lapi.obj
 0001:0000041b       _lua_pushcclosure@12       1000141b f   lapi.obj
 0001:00000420       _lua_pushlstring@12        10001420 f   lapi.obj
 0001:00000456       _lua_pushnil@4             10001456 f   lapi.obj
 0001:00000477       _lua_pushnumber@12         10001477 f   lapi.obj
 0001:000004a7       _lua_pushstring@8          100014a7 f   lapi.obj
 0001:000004d3       _lua_pushusertag@12        100014d3 f   lapi.obj
 0001:0000052b       _lua_pushvalue@8           1000152b f   lapi.obj
 0001:0000055c       _lua_rawcall@12            1000155c f   lapi.obj
 0001:0000057c       _lua_rawget@8              1000157c f   lapi.obj
 0001:000005b9       _lua_rawgeti@12            100015b9 f   lapi.obj
 0001:00000611       _lua_rawset@8              10001611 f   lapi.obj
 0001:00000660       _lua_rawseti@12            10001660 f   lapi.obj
 0001:000006ae       _lua_ref@8                 100016ae f   lapi.obj
 0001:0000073a       _lua_remove@8              1000173a f   lapi.obj
 0001:00000770       _lua_setgcthreshold@8      10001770 f   lapi.obj
 0001:00000795       _lua_setglobal@8           10001795 f   lapi.obj
 0001:000007b8       _lua_setglobals@4          100017b8 f   lapi.obj
 0001:000007ca       _lua_settable@8            100017ca f   lapi.obj
 0001:000007fc       _lua_settag@8              100017fc f   lapi.obj
 0001:00000844       _lua_settop@8              10001844 f   lapi.obj
 0001:00000867       _lua_stackspace@4          10001867 f   lapi.obj
 0001:00000876       _lua_strlen@8              10001876 f   lapi.obj
 0001:000008ab       _lua_tag@8                 100018ab f   lapi.obj
 0001:000008ca       _lua_tocfunction@8         100018ca f   lapi.obj
 0001:000008f2       _lua_tonumber@8            100018f2 f   lapi.obj
 0001:0000092f       _lua_topointer@8           1000192f f   lapi.obj
 0001:00000956       _lua_tostring@8            10001956 f   lapi.obj
 0001:0000098b       _lua_touserdata@8          1000198b f   lapi.obj
 0001:000009ad       _lua_type@8                100019ad f   lapi.obj
 0001:000009c8       _lua_typename@8            100019c8 f   lapi.obj
 0001:000009e2       _lua_unref@8               100019e2 f   lapi.obj
 0001:00000aa5       _luaL_addlstring@12        10001aa5 f   lauxlib.obj
 0001:00000ade       _luaL_addstring@8          10001ade f   lauxlib.obj
 0001:00000af9       _luaL_addvalue@4           10001af9 f   lauxlib.obj
 0001:00000b5c       _luaL_argerror@12          10001b5c f   lauxlib.obj
 0001:00000bac       _luaL_buffinit@8           10001bac f   lauxlib.obj
 0001:00000bc3       _luaL_check_lstr@12        10001bc3 f   lauxlib.obj
 0001:00000c02       _luaL_check_number@8       10001c02 f   lauxlib.obj
 0001:00000c51       _luaL_checkany@8           10001c51 f   lauxlib.obj
 0001:00000c78       _luaL_checkstack@12        10001c78 f   lauxlib.obj
 0001:00000c9f       _luaL_checktype@12         10001c9f f   lauxlib.obj
 0001:00000cbc       _luaL_findstring@8         10001cbc f   lauxlib.obj
 0001:00000cf0       _luaL_openlib@12           10001cf0 f   lauxlib.obj
 0001:00000d24       _luaL_opt_lstr@16          10001d24 f   lauxlib.obj
 0001:00000d6c       _luaL_opt_number@16        10001d6c f   lauxlib.obj
 0001:00000d93       _luaL_prepbuffer@4         10001d93 f   lauxlib.obj
 0001:00000daf       _luaL_pushresult@4         10001daf f   lauxlib.obj
 0001:00000de6       _luaL_verror               10001de6 f   lauxlib.obj
 0001:00001b65       _lua_baselibopen@4         10002b65 f   lbaselib.obj
 0001:00001bb7       _lua_minbaselibopen@4      10002bb7 f   lbaselib.obj
 0001:00001c4c       _setAlertCallback@4        10002c4c f   lbaselib.obj
 0001:00001c58       _setOutputCallback@4       10002c58 f   lbaselib.obj
 0001:00001e27       _luaK_adjuststack@8        10002e27 f   lcode.obj
 0001:00001e45       _luaK_code0@8              10002e45 f   lcode.obj
 0001:00001e59       _luaK_code1@12             10002e59 f   lcode.obj
 0001:00001e6f       _luaK_code2@16             10002e6f f   lcode.obj
 0001:000021b3       _luaK_concat@12            100031b3 f   lcode.obj
 0001:000021ec       _luaK_deltastack@8         100031ec f   lcode.obj
 0001:0000222b       _luaK_error@8              1000322b f   lcode.obj
 0001:000022cb       _luaK_getlabel@4           100032cb f   lcode.obj
 0001:00002313       _luaK_goiftrue@12          10003313 f   lcode.obj
 0001:00002334       _luaK_infix@12             10003334 f   lcode.obj
 0001:0000236b       _luaK_jump@4               1000336b f   lcode.obj
 0001:0000239f       _luaK_kstr@8               1000339f f   lcode.obj
 0001:000023b4       _luaK_lastisopen@4         100033b4 f   lcode.obj
 0001:000023dd       _luaK_number@12            100033dd f   lcode.obj
 0001:0000242b       _luaK_patchlist@12         1000342b f   lcode.obj
 0001:000024d0       _luaK_posfix@16            100034d0 f   lcode.obj
 0001:0000254a       _luaK_prefix@12            1000354a f   lcode.obj
 0001:000025c2       _luaK_setcallreturns@8     100035c2 f   lcode.obj
 0001:00002600       _luaK_storevar@8           10003600 f   lcode.obj
 0001:000026ca       _luaK_tostack@12           100036ca f   lcode.obj
 0001:00002bf4       _lua_dblibopen@4           10003bf4 f   ldblib.obj
 0001:00003025       _luaG_binerror@16          10004025 f   ldebug.obj
 0001:00003045       _luaG_getline@16           10004045 f   ldebug.obj
 0001:000030b5       _luaG_ordererror@8         100040b5 f   ldebug.obj
 0001:00003256       _luaG_typeerror@12         10004256 f   ldebug.obj
 0001:000032aa       _lua_getinfo@12            100042aa f   ldebug.obj
 0001:000033c3       _lua_getlocal@12           100043c3 f   ldebug.obj
 0001:00003408       _lua_getstack@12           10004408 f   ldebug.obj
 0001:0000342b       _lua_setcallhook@8         1000442b f   ldebug.obj
 0001:0000343c       _lua_setlinehook@8         1000443c f   ldebug.obj
 0001:0000344d       _lua_setlocal@12           1000444d f   ldebug.obj
 0001:00003678       _luaD_adjusttop@12         10004678 f   ldo.obj
 0001:000036b8       _luaD_breakrun@8           100046b8 f   ldo.obj
 0001:000036ef       _luaD_call@12              100046ef f   ldo.obj
 0001:0000384a       _luaD_callTM@16            1000484a f   ldo.obj
 0001:0000387f       _luaD_checkstack@8         1000487f f   ldo.obj
 0001:000038c6       _luaD_init@8               100048c6 f   ldo.obj
 0001:000038ff       _luaD_lineHook@16          100048ff f   ldo.obj
 0001:00003976       _luaD_runprotected@12      10004976 f   ldo.obj
 0001:000039fc       _lua_call@12               100049fc f   ldo.obj
 0001:00003a35       _lua_dobuffer@16           10004a35 f   ldo.obj
 0001:00003a8c       _lua_dofile@8              10004a8c f   ldo.obj
 0001:00003aac       _lua_dostring@8            10004aac f   ldo.obj
 0001:00003acb       _lua_error@8               10004acb f   ldo.obj
 0001:00003d12       _luaF_freeclosure@8        10004d12 f   lfunc.obj
 0001:00003d38       _luaF_freeproto@8          10004d38 f   lfunc.obj
 0001:00003d9c       _luaF_getlocalname@12      10004d9c f   lfunc.obj
 0001:00003de1       _luaF_newclosure@8         10004de1 f   lfunc.obj
 0001:00003e14       _luaF_newproto@4           10004e14 f   lfunc.obj
 0001:00003e68       _luaF_protook@12           10004e68 f   lfunc.obj
 0001:000041d8       _luaC_checkGC@4            100051d8 f   lgc.obj
 0001:000041ed       _luaC_collect@8            100051ed f   lgc.obj
 0001:00004c13       _errorfb@4                 10005c13 f   liolib.obj
 0001:0000519d       _lua_iolibopen@4           1000619d f   liolib.obj
 0001:000051b2       _lua_miniolibopen@4        100061b2 f   liolib.obj
 0001:0000564f       _luaX_checklimit@16        1000664f f   llex.obj
 0001:00005687       _luaX_error@12             10006687 f   llex.obj
 0001:000056c1       _luaX_init@4               100066c1 f   llex.obj
 0001:00005718       _luaX_lex@8                10006718 f   llex.obj
 0001:00005bd9       _luaX_setinput@16          10006bd9 f   llex.obj
 0001:00005c67       _luaX_syntaxerror@12       10006c67 f   llex.obj
 0001:00005ca5       _luaX_token2str@8          10006ca5 f   llex.obj
 0001:00006b5f       _lua_mathlibopen@4         10007b5f f   lmathlib.obj
 0001:00006be8       _luaM_growaux@28           10007be8 f   lmem.obj
 0001:00006c3c       _luaM_realloc@12           10007c3c f   lmem.obj
 0001:00006c8a       _luaO_chunkid@12           10007c8a f   lobject.obj
 0001:00006d4b       _luaO_equalObj@8           10007d4b f   lobject.obj
 0001:00006d9c       _luaO_openspace@8          10007d9c f   lobject.obj
 0001:00006dcb       _luaO_power2@4             10007dcb f   lobject.obj
 0001:00006ddf       _luaO_str2d@8              10007ddf f   lobject.obj
 0001:00006e36       _luaO_verror               10007e36 f   lobject.obj
 0001:00007b60       _luaY_parser@8             10008b60 f   lparser.obj
 0001:000086a9       _lua_print@4               100096a9 f   lprint.obj
 0001:0000875e       _lua_close@4               1000975e f   lstate.obj
 0001:000087db       _lua_open@4                100097db f   lstate.obj
 0001:000088ae       _luaS_createudata@12       100098ae f   lstring.obj
 0001:000088f8       _luaS_freeall@4            100098f8 f   lstring.obj
 0001:00008923       _luaS_init@4               10009923 f   lstring.obj
 0001:00008962       _luaS_new@8                10009962 f   lstring.obj
 0001:0000897d       _luaS_newfixed@8           1000997d f   lstring.obj
 0001:0000899a       _luaS_newlstr@12           1000999a f   lstring.obj
 0001:00008a59       _luaS_newudata@12          10009a59 f   lstring.obj
 0001:00008ab4       _luaS_resize@12            10009ab4 f   lstring.obj
 0001:00009739       _luaI_classend@8           1000a739 f   lstrlib.obj
 0001:00009797       _luaI_singlematch@12       1000a797 f   lstrlib.obj
 0001:000097e0       _lua_strlibopen@4          1000a7e0 f   lstrlib.obj
 0001:00009db1       _luaH_free@8               1000adb1 f   ltable.obj
 0001:00009de1       _luaH_get@12               1000ade1 f   ltable.obj
 0001:00009e6a       _luaH_getglobal@8          1000ae6a f   ltable.obj
 0001:00009e86       _luaH_getnum@12            1000ae86 f   ltable.obj
 0001:00009ec5       _luaH_getstr@8             1000aec5 f   ltable.obj
 0001:00009ef6       _luaH_mainposition@8       1000aef6 f   ltable.obj
 0001:00009f38       _luaH_new@8                1000af38 f   ltable.obj
 0001:00009f80       _luaH_next@12              1000af80 f   ltable.obj
 0001:00009fe9       _luaH_remove@8             1000afe9 f   ltable.obj
 0001:0000a07f       _luaH_set@12               1000b07f f   ltable.obj
 0001:0000a134       _luaH_setint@12            1000b134 f   ltable.obj
 0001:0000a162       _luaH_setstrnum@20         1000b162 f   ltable.obj
 0001:0000a3f9       _luaT_init@4               1000b3f9 f   ltm.obj
 0001:0000a43c       _luaT_realtag@8            1000b43c f   ltm.obj
 0001:0000a460       _luaT_tag@4                1000b460 f   ltm.obj
 0001:0000a47f       _luaT_validevent@8         1000b47f f   ltm.obj
 0001:0000a49f       _lua_copytagmethods@12     1000b49f f   ltm.obj
 0001:0000a4f5       _lua_gettagmethod@12       1000b4f5 f   ltm.obj
 0001:0000a55b       _lua_newtag@4              1000b55b f   ltm.obj
 0001:0000a594       _lua_settagmethod@12       1000b594 f   ltm.obj
 0001:0000ad2e       _luaU_endianess@0          1000bd2e f   lundump.obj
 0001:0000ad32       _luaU_undump@8             1000bd32 f   lundump.obj
 0001:0000aeb6       _luaV_Cclosure@12          1000beb6 f   lvm.obj
 0001:0000aed3       _luaV_Lclosure@12          1000bed3 f   lvm.obj
 0001:0000af52       _luaV_execute@12           1000bf52 f   lvm.obj
 0001:0000b98e       _luaV_getglobal@8          1000c98e f   lvm.obj
 0001:0000ba06       _luaV_gettable@8           1000ca06 f   lvm.obj
 0001:0000bacd       _luaV_lessthan@16          1000cacd f   lvm.obj
 0001:0000bc1b       _luaV_setglobal@8          1000cc1b f   lvm.obj
 0001:0000bcee       _luaV_settable@12          1000ccee f   lvm.obj
 0001:0000be13       _luaV_strconc@12           1000ce13 f   lvm.obj
 0001:0000bf7f       _luaV_tonumber@4           1000cf7f f   lvm.obj
 0001:0000bfb2       _luaV_tostring@8           1000cfb2 f   lvm.obj
 0001:0000c06a       _luaZ_Fopen@12             1000d06a f   lzio.obj
 0001:0000c097       _luaZ_mopen@16             1000d097 f   lzio.obj
 0001:0000c0c5       _luaZ_read@12              1000d0c5 f   lzio.obj
 0001:0000c118       _luaZ_sopen@12             1000d118 f   lzio.obj
 0001:0000c1bb       _luaOverload_free@4        1000d1bb f   LuaMem.obj
 0001:0000c1d6       _luaOverload_realloc@8     1000d1d6 f   LuaMem.obj
 0001:0000c223       _lua_exit@0                1000d223 f   LuaMem.obj
 0001:0000c246       _ascii_atod@4              1000d246 f   Assist:AsciiCType.obj
 0001:0000c29f       _ascii_atol@4              1000d29f f   Assist:AsciiCType.obj
 0001:0000c2d4       _ascii_strtod@8            1000d2d4 f   Assist:AsciiCType.obj
 0001:0000c2f5       _ascii_strtol@12           1000d2f5 f   Assist:AsciiCType.obj
 0001:0000c31a       _ascii_strtoul@12          1000d31a f   Assist:AsciiCType.obj
 0001:0000c33f       ??$_Allocate@D@std@@YGPADIPAD@Z 1000d33f f i Assist:pch.obj
 0001:0000c366       ??$addressof@D@std@@YGPADAAD@Z 1000d366 f i Assist:pch.obj
 0001:0000c36d       ??$construct@PADAAPAD@?$_Wrap_alloc@V?$allocator@D@std@@@std@@QAEXPAPADAAPAD@Z 1000d36d f i Assist:pch.obj
 0001:0000c380       ??$construct@PADAAPAD@?$allocator@D@std@@QAEXPAPADAAPAD@Z 1000d380 f i Assist:pch.obj
 0001:0000c393       ??$construct@PADAAPAD@?$allocator_traits@V?$allocator@D@std@@@std@@SGXAAV?$allocator@D@1@PAPADAAPAD@Z 1000d393 f i Assist:pch.obj
 0001:0000c3a6       ??$destroy@PAD@?$_Wrap_alloc@V?$allocator@D@std@@@std@@QAEXPAPAD@Z 1000d3a6 f i Assist:pch.obj
 0001:0000c3a9       ??$destroy@PAD@?$allocator@D@std@@QAEXPAPAD@Z 1000d3a9 f i Assist:pch.obj
 0001:0000c3ac       ??$destroy@PAD@?$allocator_traits@V?$allocator@D@std@@@std@@SGXAAV?$allocator@D@1@PAPAD@Z 1000d3ac f i Assist:pch.obj
 0001:0000c3af       ??$forward@AAPAD@std@@YGAAPADAAPAD@Z 1000d3af f i Assist:pch.obj
 0001:0000c3b6       ??0?$_String_alloc@$0A@U?$_String_base_types@DV?$allocator@D@std@@@std@@@std@@QAE@ABV?$allocator@D@1@@Z 1000d3b6 f i Assist:pch.obj
 0001:0000c3c3       ??0?$_String_val@U?$_Simple_types@D@std@@@std@@QAE@XZ 1000d3c3 f i Assist:pch.obj
 0001:0000c3ce       ??0?$_Wrap_alloc@V?$allocator@D@std@@@std@@QAE@XZ 1000d3ce f i Assist:pch.obj
 0001:0000c3d1       ??0?$allocator@D@std@@QAE@XZ 1000d3d1 f i Assist:pch.obj
 0001:0000c3d4       ??0?$basic_string@DU?$char_traits@D@std@@V?$allocator@D@2@@std@@QAE@PBD@Z 1000d3d4 f i Assist:pch.obj
 0001:0000c401       ??0_Generic_error_category@std@@QAE@XZ 1000d401 f i Assist:pch.obj
 0001:0000c40a       ??0_Iostream_error_category@std@@QAE@XZ 1000d40a f i Assist:pch.obj
 0001:0000c413       ??0_System_error_category@std@@QAE@XZ 1000d413 f i Assist:pch.obj
 0001:0000c41c       ??0error_category@std@@QAE@XZ 1000d41c f i Assist:pch.obj
 0001:0000c425       ??0error_condition@std@@QAE@HABVerror_category@1@@Z 1000d425 f i Assist:pch.obj
 0001:0000c437       ??1?$basic_string@DU?$char_traits@D@std@@V?$allocator@D@2@@std@@QAE@XZ 1000d437 f i Assist:pch.obj
 0001:0000c458       ??1_Generic_error_category@std@@UAE@XZ 1000d458 f i Assist:pch.obj
 0001:0000c45f       ??1_Iostream_error_category@std@@UAE@XZ 1000d45f f i Assist:pch.obj
 0001:0000c466       ??1_System_error_category@std@@UAE@XZ 1000d466 f i Assist:pch.obj
 0001:0000c46d       ??1error_category@std@@UAE@XZ 1000d46d f i Assist:pch.obj
 0001:0000c474       ??2@YAPAXIPAX@Z            1000d474 f i Assist:pch.obj
 0001:0000c479       ??3@YAXPAX0@Z              1000d479 f i Assist:pch.obj
 0001:0000c47a       ??8error_category@std@@QBE_NABV01@@Z 1000d47a f i Assist:pch.obj
 0001:0000c486       ??8error_condition@std@@QBE_NABV01@@Z 1000d486 f i Assist:pch.obj
 0001:0000c4a2       ??_E_Generic_error_category@std@@UAEPAXI@Z 1000d4a2 f i Assist:pch.obj
 0001:0000c4a2       ??_G_Generic_error_category@std@@UAEPAXI@Z 1000d4a2 f i Assist:pch.obj
 0001:0000c4bf       ??_G_Iostream_error_category@std@@UAEPAXI@Z 1000d4bf f i Assist:pch.obj
 0001:0000c4bf       ??_E_Iostream_error_category@std@@UAEPAXI@Z 1000d4bf f i Assist:pch.obj
 0001:0000c4dc       ??_E_System_error_category@std@@UAEPAXI@Z 1000d4dc f i Assist:pch.obj
 0001:0000c4dc       ??_G_System_error_category@std@@UAEPAXI@Z 1000d4dc f i Assist:pch.obj
 0001:0000c4f9       ??_Gerror_category@std@@UAEPAXI@Z 1000d4f9 f i Assist:pch.obj
 0001:0000c4f9       ??_Eerror_category@std@@UAEPAXI@Z 1000d4f9 f i Assist:pch.obj
 0001:0000c516       ?_Copy@?$basic_string@DU?$char_traits@D@std@@V?$allocator@D@2@@std@@QAEXII@Z 1000d516 f i Assist:pch.obj
 0001:0000c62b       ?_Eos@?$basic_string@DU?$char_traits@D@std@@V?$allocator@D@2@@std@@QAEXI@Z 1000d62b f i Assist:pch.obj
 0001:0000c641       ?_Getal@?$_String_alloc@$0A@U?$_String_base_types@DV?$allocator@D@std@@@std@@@std@@QBE?AU?$_Wrap_alloc@V?$allocator@D@std@@@2@XZ 1000d641 f i Assist:pch.obj
 0001:0000c648       ?_Grow@?$basic_string@DU?$char_traits@D@std@@V?$allocator@D@2@@std@@QAE_NI_N@Z 1000d648 f i Assist:pch.obj
 0001:0000c6a9       ?_Inside@?$basic_string@DU?$char_traits@D@std@@V?$allocator@D@2@@std@@QAE_NPBD@Z 1000d6a9 f i Assist:pch.obj
 0001:0000c6e1       ?_Myptr@?$_String_val@U?$_Simple_types@D@std@@@std@@QAEPADXZ 1000d6e1 f i Assist:pch.obj
 0001:0000c6ec       ?_Myptr@?$_String_val@U?$_Simple_types@D@std@@@std@@QBEPBDXZ 1000d6ec f i Assist:pch.obj
 0001:0000c6f7       ?_Tidy@?$basic_string@DU?$char_traits@D@std@@V?$allocator@D@2@@std@@QAEX_NI@Z 1000d6f7 f i Assist:pch.obj
 0001:0000c739       ?_Xlen@?$basic_string@DU?$char_traits@D@std@@V?$allocator@D@2@@std@@QBEXXZ 1000d739 f i Assist:pch.obj
 0001:0000c745       ?_Xran@?$basic_string@DU?$char_traits@D@std@@V?$allocator@D@2@@std@@QBEXXZ 1000d745 f i Assist:pch.obj
 0001:0000c751       ?allocate@?$_Wrap_alloc@V?$allocator@D@std@@@std@@QAEPADI@Z 1000d751 f i Assist:pch.obj
 0001:0000c75f       ?allocate@?$allocator@D@std@@QAEPADI@Z 1000d75f f i Assist:pch.obj
 0001:0000c76d       ?assign@?$basic_string@DU?$char_traits@D@std@@V?$allocator@D@2@@std@@QAEAAV12@ABV12@II@Z 1000d76d f i Assist:pch.obj
 0001:0000c7ff       ?assign@?$basic_string@DU?$char_traits@D@std@@V?$allocator@D@2@@std@@QAEAAV12@PBD@Z 1000d7ff f i Assist:pch.obj
 0001:0000c81c       ?assign@?$basic_string@DU?$char_traits@D@std@@V?$allocator@D@2@@std@@QAEAAV12@PBDI@Z 1000d81c f i Assist:pch.obj
 0001:0000c894       ?assign@?$char_traits@D@std@@SAXAADABD@Z 1000d894 f i Assist:pch.obj
 0001:0000c8a1       ?category@error_code@std@@QBEABVerror_category@2@XZ 1000d8a1 f i Assist:pch.obj
 0001:0000c8a5       ?category@error_condition@std@@QBEABVerror_category@2@XZ 1000d8a5 f i Assist:pch.obj
 0001:0000c8a9       ?copy@?$char_traits@D@std@@SAPADPADPBDI@Z 1000d8a9 f i Assist:pch.obj
 0001:0000c8bd       ?deallocate@?$_Wrap_alloc@V?$allocator@D@std@@@std@@QAEXPADI@Z 1000d8bd f i Assist:pch.obj
 0001:0000c8ca       ?deallocate@?$allocator@D@std@@QAEXPADI@Z 1000d8ca f i Assist:pch.obj
 0001:0000c8d7       ?default_error_condition@_System_error_category@std@@UBE?AVerror_condition@2@H@Z 1000d8d7 f i Assist:pch.obj
 0001:0000c902       ?default_error_condition@error_category@std@@UBE?AVerror_condition@2@H@Z 1000d902 f i Assist:pch.obj
 0001:0000c912       ?equivalent@error_category@std@@UBE_NABVerror_code@2@H@Z 1000d912 f i Assist:pch.obj
 0001:0000c92d       ?equivalent@error_category@std@@UBE_NHABVerror_condition@2@@Z 1000d92d f i Assist:pch.obj
 0001:0000c94c       ?erase@?$basic_string@DU?$char_traits@D@std@@V?$allocator@D@2@@std@@QAEAAV12@I@Z 1000d94c f i Assist:pch.obj
 0001:0000c978       ?erase@?$basic_string@DU?$char_traits@D@std@@V?$allocator@D@2@@std@@QAEAAV12@II@Z 1000d978 f i Assist:pch.obj
 0001:0000c9f9       ?generic_category@std@@YGABVerror_category@1@XZ 1000d9f9 f i Assist:pch.obj
 0001:0000c9ff       ?length@?$char_traits@D@std@@SAIPBD@Z 1000d9ff f i Assist:pch.obj
 0001:0000ca13       ?max_size@?$_Wrap_alloc@V?$allocator@D@std@@@std@@QBEIXZ 1000da13 f i Assist:pch.obj
 0001:0000ca17       ?max_size@?$allocator@D@std@@QBEIXZ 1000da17 f i Assist:pch.obj
 0001:0000ca1b       ?max_size@?$allocator_traits@V?$allocator@D@std@@@std@@SGIABV?$allocator@D@2@@Z 1000da1b f i Assist:pch.obj
 0001:0000ca21       ?max_size@?$basic_string@DU?$char_traits@D@std@@V?$allocator@D@2@@std@@QBEIXZ 1000da21 f i Assist:pch.obj
 0001:0000ca25       ?message@_Generic_error_category@std@@UBE?AV?$basic_string@DU?$char_traits@D@std@@V?$allocator@D@2@@2@H@Z 1000da25 f i Assist:pch.obj
 0001:0000ca51       ?message@_Iostream_error_category@std@@UBE?AV?$basic_string@DU?$char_traits@D@std@@V?$allocator@D@2@@2@H@Z 1000da51 f i Assist:pch.obj
 0001:0000ca80       ?message@_System_error_category@std@@UBE?AV?$basic_string@DU?$char_traits@D@std@@V?$allocator@D@2@@2@H@Z 1000da80 f i Assist:pch.obj
 0001:0000caac       ?move@?$char_traits@D@std@@SAPADPADPBDI@Z 1000daac f i Assist:pch.obj
 0001:0000cac1       ?name@_Generic_error_category@std@@UBEPBDXZ 1000dac1 f i Assist:pch.obj
 0001:0000cac7       ?name@_Iostream_error_category@std@@UBEPBDXZ 1000dac7 f i Assist:pch.obj
 0001:0000cacd       ?name@_System_error_category@std@@UBEPBDXZ 1000dacd f i Assist:pch.obj
 0001:0000cad3       ?size@?$basic_string@DU?$char_traits@D@std@@V?$allocator@D@2@@std@@QBEIXZ 1000dad3 f i Assist:pch.obj
 0001:0000cad7       ?system_category@std@@YGABVerror_category@1@XZ 1000dad7 f i Assist:pch.obj
 0001:0000cadd       ?value@error_code@std@@QBEHXZ 1000dadd f i Assist:pch.obj
 0001:0000cae0       ?value@error_condition@std@@QBEHXZ 1000dae0 f i Assist:pch.obj
 0001:0000cae4       ?dbFatalfAux@@YAXPBDZZ     1000dae4 f   Debug:Debug.dll
 0001:0000caea       ?MemPoolAlloc@@YGPAXPAU_HMEMPOOL@@I@Z 1000daea f   Memory:Memory.dll
 0001:0000caf0       ?MemPoolFree@@YGXPAU_HMEMPOOL@@PAX@Z 1000daf0 f   Memory:Memory.dll
 0001:0000caf6       ??0MemoryPoolObj@@QAE@PBDI@Z 1000daf6 f   Memory:Memory.dll
 0001:0000cafc       ??1MemoryPoolObj@@QAE@XZ   1000dafc f   Memory:Memory.dll
 0001:0000cb02       ?_Xbad_alloc@std@@YAXXZ    1000db02 f   msvcprt:MSVCP110.dll
 0001:0000cb08       ?_Xlength_error@std@@YAXPBD@Z 1000db08 f   msvcprt:MSVCP110.dll
 0001:0000cb0e       ?_Xout_of_range@std@@YAXPBD@Z 1000db0e f   msvcprt:MSVCP110.dll
 0001:0000cb14       ??0id@locale@std@@QAE@I@Z  1000db14 f   msvcprt:MSVCP110.dll
 0001:0000cb1a       ?_Syserror_map@std@@YAPBDH@Z 1000db1a f   msvcprt:MSVCP110.dll
 0001:0000cb20       ?_Winerror_map@std@@YAPBDH@Z 1000db20 f   msvcprt:MSVCP110.dll
 0001:0000cb26       _strlen                    1000db26 f   MSVCRT:MSVCR110.dll
 0001:0000cb30       _sprintf                   1000db30 f   MSVCRT:MSVCR110.dll
 0001:0000cb36       _vsprintf                  1000db36 f   MSVCRT:MSVCR110.dll
 0001:0000cb3c       _memcpy                    1000db3c f   MSVCRT:MSVCR110.dll
 0001:0000cb42       _strcmp                    1000db42 f   MSVCRT:MSVCR110.dll
 0001:0000cb48       _strchr                    1000db48 f   MSVCRT:MSVCR110.dll
 0001:0000cb50       __ftol2_sse                1000db50 f   MSVCRT:ftol2.obj
 0001:0000cb59       __ftol2_pentium4           1000db59 f   MSVCRT:ftol2.obj
 0001:0000cb6c       __ftol2_sse_excpt          1000db6c f   MSVCRT:ftol2.obj
 0001:0000cb86       __ftol2                    1000db86 f   MSVCRT:ftol2.obj
 0001:0000cbfc       _abs                       1000dbfc f   MSVCRT:MSVCR110.dll
 0001:0000cc02       _longjmp                   1000dc02 f   MSVCRT:MSVCR110.dll
 0001:0000cc08       ___iob_func                1000dc08 f   MSVCRT:MSVCR110.dll
 0001:0000cc0e       _fclose                    1000dc0e f   MSVCRT:MSVCR110.dll
 0001:0000cc14       _fgetc                     1000dc14 f   MSVCRT:MSVCR110.dll
 0001:0000cc1a       _fopen                     1000dc1a f   MSVCRT:MSVCR110.dll
 0001:0000cc20       _freopen                   1000dc20 f   MSVCRT:MSVCR110.dll
 0001:0000cc26       _ungetc                    1000dc26 f   MSVCRT:MSVCR110.dll
 0001:0000cc2c       _strncpy                   1000dc2c f   MSVCRT:MSVCR110.dll
 0001:0000cc32       __setjmp3                  1000dc32 f   MSVCRT:MSVCR110.dll
 0001:0000cc38       _fflush                    1000dc38 f   MSVCRT:MSVCR110.dll
 0001:0000cc3e       _fgets                     1000dc3e f   MSVCRT:MSVCR110.dll
 0001:0000cc44       _fprintf                   1000dc44 f   MSVCRT:MSVCR110.dll
 0001:0000cc4a       _fread                     1000dc4a f   MSVCRT:MSVCR110.dll
 0001:0000cc50       _fscanf                    1000dc50 f   MSVCRT:MSVCR110.dll
 0001:0000cc56       _fseek                     1000dc56 f   MSVCRT:MSVCR110.dll
 0001:0000cc5c       _ftell                     1000dc5c f   MSVCRT:MSVCR110.dll
 0001:0000cc62       _fwrite                    1000dc62 f   MSVCRT:MSVCR110.dll
 0001:0000cc68       _remove                    1000dc68 f   MSVCRT:MSVCR110.dll
 0001:0000cc6e       _rename                    1000dc6e f   MSVCRT:MSVCR110.dll
 0001:0000cc74       _tmpnam                    1000dc74 f   MSVCRT:MSVCR110.dll
 0001:0000cc7a       __errno                    1000dc7a f   MSVCRT:MSVCR110.dll
 0001:0000cc80       _getenv                    1000dc80 f   MSVCRT:MSVCR110.dll
 0001:0000cc86       _system                    1000dc86 f   MSVCRT:MSVCR110.dll
 0001:0000cc8c       _strerror                  1000dc8c f   MSVCRT:MSVCR110.dll
 0001:0000cc92       _clock                     1000dc92 f   MSVCRT:MSVCR110.dll
 0001:0000cc98       _strftime                  1000dc98 f   MSVCRT:MSVCR110.dll
 0001:0000cc9e       __localtime64              1000dc9e f   MSVCRT:MSVCR110.dll
 0001:0000cca4       __time64                   1000dca4 f   MSVCRT:MSVCR110.dll
 0001:0000ccaa       _strcpy                    1000dcaa f   MSVCRT:MSVCR110.dll
 0001:0000ccb0       _rand                      1000dcb0 f   MSVCRT:MSVCR110.dll
 0001:0000ccb6       _srand                     1000dcb6 f   MSVCRT:MSVCR110.dll
 0001:0000ccbc       _acos                      1000dcbc f   MSVCRT:MSVCR110.dll
 0001:0000ccc2       _asin                      1000dcc2 f   MSVCRT:MSVCR110.dll
 0001:0000ccc8       _atan                      1000dcc8 f   MSVCRT:MSVCR110.dll
 0001:0000ccce       _atan2                     1000dcce f   MSVCRT:MSVCR110.dll
 0001:0000ccd4       _cos                       1000dcd4 f   MSVCRT:MSVCR110.dll
 0001:0000ccda       _exp                       1000dcda f   MSVCRT:MSVCR110.dll
 0001:0000cce0       _fabs                      1000dce0 f   MSVCRT:MSVCR110.dll
 0001:0000cce6       _fmod                      1000dce6 f   MSVCRT:MSVCR110.dll
 0001:0000ccec       _log                       1000dcec f   MSVCRT:MSVCR110.dll
 0001:0000ccf2       _log10                     1000dcf2 f   MSVCRT:MSVCR110.dll
 0001:0000ccf8       _pow                       1000dcf8 f   MSVCRT:MSVCR110.dll
 0001:0000ccfe       _sin                       1000dcfe f   MSVCRT:MSVCR110.dll
 0001:0000cd04       _tan                       1000dd04 f   MSVCRT:MSVCR110.dll
 0001:0000cd0a       _sqrt                      1000dd0a f   MSVCRT:MSVCR110.dll
 0001:0000cd10       _ceil                      1000dd10 f   MSVCRT:MSVCR110.dll
 0001:0000cd16       _floor                     1000dd16 f   MSVCRT:MSVCR110.dll
 0001:0000cd1c       _frexp                     1000dd1c f   MSVCRT:MSVCR110.dll
 0001:0000cd22       _ldexp                     1000dd22 f   MSVCRT:MSVCR110.dll
 0001:0000cd28       _strcspn                   1000dd28 f   MSVCRT:MSVCR110.dll
 0001:0000cd2e       _memcmp                    1000dd2e f   MSVCRT:MSVCR110.dll
 0001:0000cd34       _toupper                   1000dd34 f   MSVCRT:MSVCR110.dll
 0001:0000cd3a       _tolower                   1000dd3a f   MSVCRT:MSVCR110.dll
 0001:0000cd40       _memchr                    1000dd40 f   MSVCRT:MSVCR110.dll
 0001:0000cd46       _strpbrk                   1000dd46 f   MSVCRT:MSVCR110.dll
 0001:0000cd4c       _strcoll                   1000dd4c f   MSVCRT:MSVCR110.dll
 0001:0000cd52       _feof                      1000dd52 f   MSVCRT:MSVCR110.dll
 0001:0000cd58       ___atonexitinit            1000dd58 f   MSVCRT:atonexit.obj
 0001:0000cd94       __onexit                   1000dd94 f   MSVCRT:atonexit.obj
 0001:0000ce39       _atexit                    1000de39 f   MSVCRT:atonexit.obj
 0001:0000ce9a       _NtCurrentTeb              1000de9a f i MSVCRT:crtdll.obj
 0001:0000cea1       __CRT_INIT@12              1000dea1 f   MSVCRT:crtdll.obj
 0001:0000d096       __DllMainCRTStartup@12     1000e096 f   MSVCRT:crtdll.obj
 0001:0000d1ec       _strtod                    1000e1ec f   MSVCRT:MSVCR110.dll
 0001:0000d1f2       _strtol                    1000e1f2 f   MSVCRT:MSVCR110.dll
 0001:0000d1f8       _strtoul                   1000e1f8 f   MSVCRT:MSVCR110.dll
 0001:0000d1fe       _setlocale                 1000e1fe f   MSVCRT:MSVCR110.dll
 0001:0000d204       __purecall                 1000e204 f   MSVCRT:MSVCR110.dll
 0001:0000d20a       ??2@YAPAXI@Z               1000e20a f   MSVCRT:MSVCR110.dll
 0001:0000d210       ??3@YAXPAX@Z               1000e210 f   MSVCRT:MSVCR110.dll
 0001:0000d216       _memmove                   1000e216 f   MSVCRT:MSVCR110.dll
 0001:0000d21c       __CxxThrowException@8      1000e21c f   MSVCRT:MSVCR110.dll
 0001:0000d224       __EH_prolog                1000e224 f   MSVCRT:ehprolog.obj
 0001:0000d244       ___CxxFrameHandler3        1000e244 f   MSVCRT:MSVCR110.dll
 0001:0000d24a       ??0type_info@@AAE@ABV0@@Z  1000e24a f   MSVCRT:ti_inst.obj
 0001:0000d255       ??4type_info@@AAEAAV0@ABV0@@Z 1000e255 f   MSVCRT:ti_inst.obj
 0001:0000d25a       ??_Etype_info@@UAEPAXI@Z   1000e25a f i MSVCRT:ti_inst.obj
 0001:0000d2a4       ___isa_available_init      1000e2a4 f   MSVCRT:cpu_disp.obj
 0001:0000d3de       __lock                     1000e3de f   MSVCRT:MSVCR110.dll
 0001:0000d3e4       __unlock                   1000e3e4 f   MSVCRT:MSVCR110.dll
 0001:0000d3ea       __calloc_crt               1000e3ea f   MSVCRT:MSVCR110.dll
 0001:0000d3f0       ___dllonexit               1000e3f0 f   MSVCRT:MSVCR110.dll
 0001:0000d400       __SEH_prolog4              1000e400 f   MSVCRT:sehprolg4.obj
 0001:0000d445       __SEH_epilog4              1000e445 f   MSVCRT:sehprolg4.obj
 0001:0000d459       __except_handler4          1000e459 f   MSVCRT:chandler4gs.obj
 0001:0000d47c       ___CppXcptFilter           1000e47c f   MSVCRT:MSVCR110.dll
 0001:0000d482       __amsg_exit                1000e482 f   MSVCRT:MSVCR110.dll
 0001:0000d490       __FindPESection            1000e490 f   MSVCRT:pesect.obj
 0001:0000d4e0       __IsNonwritableInCurrentImage 1000e4e0 f   MSVCRT:pesect.obj
 0001:0000d5a0       __ValidateImageBase        1000e5a0 f   MSVCRT:pesect.obj
 0001:0000d5d2       _free                      1000e5d2 f   MSVCRT:MSVCR110.dll
 0001:0000d5d8       ___security_init_cookie    1000e5d8 f   MSVCRT:gs_support.obj
 0001:0000d672       _DllMain@12                1000e672 f   MSVCRT:dllmain.obj
 0001:0000d694       __malloc_crt               1000e694 f   MSVCRT:MSVCR110.dll
 0001:0000d69a       __RTC_Initialize           1000e69a f   MSVCRT:initsect.obj
 0001:0000d6ba       __RTC_Terminate            1000e6ba f   MSVCRT:initsect.obj
 0001:0000d6da       __initterm                 1000e6da f   MSVCRT:MSVCR110.dll
 0001:0000d6e0       __initterm_e               1000e6e0 f   MSVCRT:MSVCR110.dll
 0001:0000d6e6       ___clean_type_info_names   1000e6e6 f   MSVCRT:tncleanup.obj
 0001:0000d6f2       ??_M@YGXPAXIHP6EX0@Z@Z     1000e6f2 f   MSVCRT:ehvecdtr.obj
 0001:0000d77a       ?__ArrayUnwind@@YGXPAXIHP6EX0@Z@Z 1000e77a f   MSVCRT:ehvecdtr.obj
 0001:0000d7d8       ??1type_info@@UAE@XZ       1000e7d8 f   MSVCRT:MSVCR110.dll
 0001:0000d7de       @__security_check_cookie@4 1000e7de f   MSVCRT:secchk.obj
 0001:0000d7ee       __except_handler4_common   1000e7ee f   MSVCRT:MSVCR110.dll
 0001:0000d7f4       ___clean_type_info_names_internal 1000e7f4 f   MSVCRT:MSVCR110.dll
 0001:0000d7fa       ?terminate@@YAXXZ          1000e7fa f   MSVCRT:MSVCR110.dll
 0001:0000d800       ___raise_securityfailure   1000e800 f   MSVCRT:gs_report.obj
 0001:0000d83d       ___report_gsfailure        1000e83d f   MSVCRT:gs_report.obj
 0001:0000d936       ___report_rangecheckfailure 1000e936 f   MSVCRT:gs_report.obj
 0001:0000d942       ___report_securityfailure  1000e942 f   MSVCRT:gs_report.obj
 0001:0000da10       ___report_securityfailureEx 1000ea10 f   MSVCRT:gs_report.obj
 0001:0000db24       __crt_debugger_hook        1000eb24 f   MSVCRT:MSVCR110.dll
 0001:0000db2a       ___crtUnhandledException   1000eb2a f   MSVCRT:MSVCR110.dll
 0001:0000db30       ___crtTerminateProcess     1000eb30 f   MSVCRT:MSVCR110.dll
 0001:0000db36       _EncodePointer@4           1000eb36 f   kernel32:KERNEL32.dll
 0001:0000db3c       _DecodePointer@4           1000eb3c f   kernel32:KERNEL32.dll
 0001:0000db42       _IsProcessorFeaturePresent@4 1000eb42 f   kernel32:KERNEL32.dll
 0001:0000db48       _QueryPerformanceCounter@4 1000eb48 f   kernel32:KERNEL32.dll
 0001:0000db4e       _GetCurrentProcessId@0     1000eb4e f   kernel32:KERNEL32.dll
 0001:0000db54       _GetCurrentThreadId@0      1000eb54 f   kernel32:KERNEL32.dll
 0001:0000db5a       _GetSystemTimeAsFileTime@4 1000eb5a f   kernel32:KERNEL32.dll
 0001:0000db60       _DisableThreadLibraryCalls@4 1000eb60 f   kernel32:KERNEL32.dll
 0001:0000db66       _IsDebuggerPresent@0       1000eb66 f   kernel32:KERNEL32.dll
 0002:00000000       __imp_?g_dbFilename@@3PBDB 1000f000     Debug:Debug.dll
 0002:00000004       __imp_?g_dbLineNum@@3KA    1000f004     Debug:Debug.dll
 0002:00000008       __imp_?dbFatalfAux@@YAXPBDZZ 1000f008     Debug:Debug.dll
 0002:0000000c       \177Debug_NULL_THUNK_DATA  1000f00c     Debug:Debug.dll
 0002:00000010       __imp__IsDebuggerPresent@0 1000f010     kernel32:KERNEL32.dll
 0002:00000014       __imp__DisableThreadLibraryCalls@4 1000f014     kernel32:KERNEL32.dll
 0002:00000018       __imp__GetSystemTimeAsFileTime@4 1000f018     kernel32:KERNEL32.dll
 0002:0000001c       __imp__GetCurrentThreadId@0 1000f01c     kernel32:KERNEL32.dll
 0002:00000020       __imp__GetCurrentProcessId@0 1000f020     kernel32:KERNEL32.dll
 0002:00000024       __imp__QueryPerformanceCounter@4 1000f024     kernel32:KERNEL32.dll
 0002:00000028       __imp__IsProcessorFeaturePresent@4 1000f028     kernel32:KERNEL32.dll
 0002:0000002c       __imp__DecodePointer@4     1000f02c     kernel32:KERNEL32.dll
 0002:00000030       __imp__EncodePointer@4     1000f030     kernel32:KERNEL32.dll
 0002:00000034       \177KERNEL32_NULL_THUNK_DATA 1000f034     kernel32:KERNEL32.dll
 0002:00000038       __imp_?_Winerror_map@std@@YAPBDH@Z 1000f038     msvcprt:MSVCP110.dll
 0002:0000003c       __imp_?_Xlength_error@std@@YAXPBD@Z 1000f03c     msvcprt:MSVCP110.dll
 0002:00000040       __imp_?_Xout_of_range@std@@YAXPBD@Z 1000f040     msvcprt:MSVCP110.dll
 0002:00000044       __imp_??0id@locale@std@@QAE@I@Z 1000f044     msvcprt:MSVCP110.dll
 0002:00000048       __imp_?_Xbad_alloc@std@@YAXXZ 1000f048     msvcprt:MSVCP110.dll
 0002:0000004c       __imp_?_Syserror_map@std@@YAPBDH@Z 1000f04c     msvcprt:MSVCP110.dll
 0002:00000050       \177MSVCP110_NULL_THUNK_DATA 1000f050     msvcprt:MSVCP110.dll
 0002:00000054       __imp__strchr              1000f054     MSVCRT:MSVCR110.dll
 0002:00000058       __imp__abs                 1000f058     MSVCRT:MSVCR110.dll
 0002:0000005c       __imp__longjmp             1000f05c     MSVCRT:MSVCR110.dll
 0002:00000060       __imp____iob_func          1000f060     MSVCRT:MSVCR110.dll
 0002:00000064       __imp__fclose              1000f064     MSVCRT:MSVCR110.dll
 0002:00000068       __imp__fgetc               1000f068     MSVCRT:MSVCR110.dll
 0002:0000006c       __imp__fopen               1000f06c     MSVCRT:MSVCR110.dll
 0002:00000070       __imp__freopen             1000f070     MSVCRT:MSVCR110.dll
 0002:00000074       __imp__ungetc              1000f074     MSVCRT:MSVCR110.dll
 0002:00000078       __imp__strncpy             1000f078     MSVCRT:MSVCR110.dll
 0002:0000007c       __imp___setjmp3            1000f07c     MSVCRT:MSVCR110.dll
 0002:00000080       __imp__fflush              1000f080     MSVCRT:MSVCR110.dll
 0002:00000084       __imp__fgets               1000f084     MSVCRT:MSVCR110.dll
 0002:00000088       __imp__fprintf             1000f088     MSVCRT:MSVCR110.dll
 0002:0000008c       __imp__fread               1000f08c     MSVCRT:MSVCR110.dll
 0002:00000090       __imp__fscanf              1000f090     MSVCRT:MSVCR110.dll
 0002:00000094       __imp__fseek               1000f094     MSVCRT:MSVCR110.dll
 0002:00000098       __imp__ftell               1000f098     MSVCRT:MSVCR110.dll
 0002:0000009c       __imp__fwrite              1000f09c     MSVCRT:MSVCR110.dll
 0002:000000a0       __imp__remove              1000f0a0     MSVCRT:MSVCR110.dll
 0002:000000a4       __imp__rename              1000f0a4     MSVCRT:MSVCR110.dll
 0002:000000a8       __imp__tmpnam              1000f0a8     MSVCRT:MSVCR110.dll
 0002:000000ac       __imp___errno              1000f0ac     MSVCRT:MSVCR110.dll
 0002:000000b0       __imp__getenv              1000f0b0     MSVCRT:MSVCR110.dll
 0002:000000b4       __imp__system              1000f0b4     MSVCRT:MSVCR110.dll
 0002:000000b8       __imp__strerror            1000f0b8     MSVCRT:MSVCR110.dll
 0002:000000bc       __imp__clock               1000f0bc     MSVCRT:MSVCR110.dll
 0002:000000c0       __imp__strftime            1000f0c0     MSVCRT:MSVCR110.dll
 0002:000000c4       __imp___localtime64        1000f0c4     MSVCRT:MSVCR110.dll
 0002:000000c8       __imp___time64             1000f0c8     MSVCRT:MSVCR110.dll
 0002:000000cc       __imp__strcpy              1000f0cc     MSVCRT:MSVCR110.dll
 0002:000000d0       __imp__rand                1000f0d0     MSVCRT:MSVCR110.dll
 0002:000000d4       __imp__srand               1000f0d4     MSVCRT:MSVCR110.dll
 0002:000000d8       __imp__acos                1000f0d8     MSVCRT:MSVCR110.dll
 0002:000000dc       __imp__asin                1000f0dc     MSVCRT:MSVCR110.dll
 0002:000000e0       __imp__atan                1000f0e0     MSVCRT:MSVCR110.dll
 0002:000000e4       __imp__atan2               1000f0e4     MSVCRT:MSVCR110.dll
 0002:000000e8       __imp__cos                 1000f0e8     MSVCRT:MSVCR110.dll
 0002:000000ec       __imp__exp                 1000f0ec     MSVCRT:MSVCR110.dll
 0002:000000f0       __imp__strcmp              1000f0f0     MSVCRT:MSVCR110.dll
 0002:000000f4       __imp__fmod                1000f0f4     MSVCRT:MSVCR110.dll
 0002:000000f8       __imp__log                 1000f0f8     MSVCRT:MSVCR110.dll
 0002:000000fc       __imp__log10               1000f0fc     MSVCRT:MSVCR110.dll
 0002:00000100       __imp__memcpy              1000f100     MSVCRT:MSVCR110.dll
 0002:00000104       __imp__sin                 1000f104     MSVCRT:MSVCR110.dll
 0002:00000108       __imp__tan                 1000f108     MSVCRT:MSVCR110.dll
 0002:0000010c       __imp__sqrt                1000f10c     MSVCRT:MSVCR110.dll
 0002:00000110       __imp__ceil                1000f110     MSVCRT:MSVCR110.dll
 0002:00000114       __imp__floor               1000f114     MSVCRT:MSVCR110.dll
 0002:00000118       __imp__frexp               1000f118     MSVCRT:MSVCR110.dll
 0002:0000011c       __imp__ldexp               1000f11c     MSVCRT:MSVCR110.dll
 0002:00000120       __imp__strcspn             1000f120     MSVCRT:MSVCR110.dll
 0002:00000124       __imp__memcmp              1000f124     MSVCRT:MSVCR110.dll
 0002:00000128       __imp__toupper             1000f128     MSVCRT:MSVCR110.dll
 0002:0000012c       __imp__tolower             1000f12c     MSVCRT:MSVCR110.dll
 0002:00000130       __imp__memchr              1000f130     MSVCRT:MSVCR110.dll
 0002:00000134       __imp__strpbrk             1000f134     MSVCRT:MSVCR110.dll
 0002:00000138       __imp__strcoll             1000f138     MSVCRT:MSVCR110.dll
 0002:0000013c       __imp__feof                1000f13c     MSVCRT:MSVCR110.dll
 0002:00000140       __imp__strtod              1000f140     MSVCRT:MSVCR110.dll
 0002:00000144       __imp__strtol              1000f144     MSVCRT:MSVCR110.dll
 0002:00000148       __imp__strtoul             1000f148     MSVCRT:MSVCR110.dll
 0002:0000014c       __imp__setlocale           1000f14c     MSVCRT:MSVCR110.dll
 0002:00000150       __imp___HUGE               1000f150     MSVCRT:MSVCR110.dll
 0002:00000154       __imp___purecall           1000f154     MSVCRT:MSVCR110.dll
 0002:00000158       __imp_??2@YAPAXI@Z         1000f158     MSVCRT:MSVCR110.dll
 0002:0000015c       __imp_??3@YAXPAX@Z         1000f15c     MSVCRT:MSVCR110.dll
 0002:00000160       __imp__memmove             1000f160     MSVCRT:MSVCR110.dll
 0002:00000164       __imp___CxxThrowException@8 1000f164     MSVCRT:MSVCR110.dll
 0002:00000168       __imp____CxxFrameHandler3  1000f168     MSVCRT:MSVCR110.dll
 0002:0000016c       __imp___lock               1000f16c     MSVCRT:MSVCR110.dll
 0002:00000170       __imp___unlock             1000f170     MSVCRT:MSVCR110.dll
 0002:00000174       __imp___calloc_crt         1000f174     MSVCRT:MSVCR110.dll
 0002:00000178       __imp____dllonexit         1000f178     MSVCRT:MSVCR110.dll
 0002:0000017c       __imp___onexit             1000f17c     MSVCRT:MSVCR110.dll
 0002:00000180       __imp____CppXcptFilter     1000f180     MSVCRT:MSVCR110.dll
 0002:00000184       __imp___amsg_exit          1000f184     MSVCRT:MSVCR110.dll
 0002:00000188       __imp__free                1000f188     MSVCRT:MSVCR110.dll
 0002:0000018c       __imp___malloc_crt         1000f18c     MSVCRT:MSVCR110.dll
 0002:00000190       __imp___initterm           1000f190     MSVCRT:MSVCR110.dll
 0002:00000194       __imp___initterm_e         1000f194     MSVCRT:MSVCR110.dll
 0002:00000198       __imp_??1type_info@@UAE@XZ 1000f198     MSVCRT:MSVCR110.dll
 0002:0000019c       __imp___except_handler4_common 1000f19c     MSVCRT:MSVCR110.dll
 0002:000001a0       __imp____clean_type_info_names_internal 1000f1a0     MSVCRT:MSVCR110.dll
 0002:000001a4       __imp_?terminate@@YAXXZ    1000f1a4     MSVCRT:MSVCR110.dll
 0002:000001a8       __imp___crt_debugger_hook  1000f1a8     MSVCRT:MSVCR110.dll
 0002:000001ac       __imp____crtUnhandledException 1000f1ac     MSVCRT:MSVCR110.dll
 0002:000001b0       __imp____crtTerminateProcess 1000f1b0     MSVCRT:MSVCR110.dll
 0002:000001b4       __imp__vsprintf            1000f1b4     MSVCRT:MSVCR110.dll
 0002:000001b8       __imp__sprintf             1000f1b8     MSVCRT:MSVCR110.dll
 0002:000001bc       __imp__strlen              1000f1bc     MSVCRT:MSVCR110.dll
 0002:000001c0       __imp__pow                 1000f1c0     MSVCRT:MSVCR110.dll
 0002:000001c4       __imp__fabs                1000f1c4     MSVCRT:MSVCR110.dll
 0002:000001c8       \177MSVCR110_NULL_THUNK_DATA 1000f1c8     MSVCRT:MSVCR110.dll
 0002:000001cc       __imp_??0MemoryPoolObj@@QAE@PBDI@Z 1000f1cc     Memory:Memory.dll
 0002:000001d0       __imp_?MemPoolFree@@YGXPAU_HMEMPOOL@@PAX@Z 1000f1d0     Memory:Memory.dll
 0002:000001d4       __imp_?MemPoolAlloc@@YGPAXPAU_HMEMPOOL@@I@Z 1000f1d4     Memory:Memory.dll
 0002:000001d8       __imp_??1MemoryPoolObj@@QAE@XZ 1000f1d8     Memory:Memory.dll
 0002:000001dc       \177Memory_NULL_THUNK_DATA 1000f1dc     Memory:Memory.dll
 0002:000001e0       ___xc_a                    1000f1e0     MSVCRT:cinitexe.obj
 0002:000001fc       ___xc_z                    1000f1fc     MSVCRT:cinitexe.obj
 0002:00000200       ___xi_a                    1000f200     MSVCRT:cinitexe.obj
 0002:00000210       ___xi_z                    1000f210     MSVCRT:cinitexe.obj
 0002:00000258       ?is_signed@?$numeric_limits@E@std@@2_NB 1000f258     pch.obj
 0002:0000025c       ?digits@?$numeric_limits@E@std@@2HB 1000f25c     pch.obj
 0002:00000260       ?digits10@?$numeric_limits@E@std@@2HB 1000f260     pch.obj
 0002:00000264       ?is_signed@?$numeric_limits@F@std@@2_NB 1000f264     pch.obj
 0002:00000268       ?digits@?$numeric_limits@F@std@@2HB 1000f268     pch.obj
 0002:0000026c       ?digits10@?$numeric_limits@F@std@@2HB 1000f26c     pch.obj
 0002:00000270       ?value@?$integral_constant@I$0A@@std@@2IB 1000f270     pch.obj
 0002:00000274       ?is_signed@?$numeric_limits@G@std@@2_NB 1000f274     pch.obj
 0002:00000278       ?digits@?$numeric_limits@G@std@@2HB 1000f278     pch.obj
 0002:0000027c       ?digits10@?$numeric_limits@G@std@@2HB 1000f27c     pch.obj
 0002:00000280       ?is_signed@?$numeric_limits@H@std@@2_NB 1000f280     pch.obj
 0002:00000284       ?digits@?$numeric_limits@H@std@@2HB 1000f284     pch.obj
 0002:00000288       ?digits10@?$numeric_limits@H@std@@2HB 1000f288     pch.obj
 0002:0000028c       ?is_signed@?$numeric_limits@I@std@@2_NB 1000f28c     pch.obj
 0002:00000290       ?digits@?$numeric_limits@I@std@@2HB 1000f290     pch.obj
 0002:00000294       ?digits10@?$numeric_limits@I@std@@2HB 1000f294     pch.obj
 0002:00000298       ?is_signed@?$numeric_limits@J@std@@2_NB 1000f298     pch.obj
 0002:0000029c       ?digits@?$numeric_limits@J@std@@2HB 1000f29c     pch.obj
 0002:000002a0       ?digits10@?$numeric_limits@J@std@@2HB 1000f2a0     pch.obj
 0002:000002a4       ?value@?$_Sizeof@U_Nil@std@@U12@U12@U12@U12@U12@U12@U12@@std@@2IB 1000f2a4     pch.obj
 0002:000002a8       ?is_signed@?$numeric_limits@K@std@@2_NB 1000f2a8     pch.obj
 0002:000002ac       ?digits@?$numeric_limits@K@std@@2HB 1000f2ac     pch.obj
 0002:000002b0       ?digits10@?$numeric_limits@K@std@@2HB 1000f2b0     pch.obj
 0002:000002b4       ?is_signed@?$numeric_limits@_J@std@@2_NB 1000f2b4     pch.obj
 0002:000002b8       ?digits@?$numeric_limits@_J@std@@2HB 1000f2b8     pch.obj
 0002:000002bc       ?digits10@?$numeric_limits@_J@std@@2HB 1000f2bc     pch.obj
 0002:000002c0       ?is_signed@?$numeric_limits@_K@std@@2_NB 1000f2c0     pch.obj
 0002:000002c4       ?digits@?$numeric_limits@_K@std@@2HB 1000f2c4     pch.obj
 0002:000002c8       ?digits10@?$numeric_limits@_K@std@@2HB 1000f2c8     pch.obj
 0002:000002cc       ?value@?$integral_constant@_N$0A@@std@@2_NB 1000f2cc     pch.obj
 0002:000002cd       ?value@?$integral_constant@_N$00@std@@2_NB 1000f2cd     pch.obj
 0002:000002d0       ?digits@?$numeric_limits@M@std@@2HB 1000f2d0     pch.obj
 0002:000002d4       ?digits10@?$numeric_limits@M@std@@2HB 1000f2d4     pch.obj
 0002:000002d8       ?max_digits10@?$numeric_limits@M@std@@2HB 1000f2d8     pch.obj
 0002:000002dc       ?max_exponent@?$numeric_limits@M@std@@2HB 1000f2dc     pch.obj
 0002:000002e0       ?max_exponent10@?$numeric_limits@M@std@@2HB 1000f2e0     pch.obj
 0002:000002e4       ?min_exponent@?$numeric_limits@M@std@@2HB 1000f2e4     pch.obj
 0002:000002e8       ?min_exponent10@?$numeric_limits@M@std@@2HB 1000f2e8     pch.obj
 0002:000002ec       ?digits@?$numeric_limits@N@std@@2HB 1000f2ec     pch.obj
 0002:000002f0       ?digits10@?$numeric_limits@N@std@@2HB 1000f2f0     pch.obj
 0002:000002f4       ?max_digits10@?$numeric_limits@N@std@@2HB 1000f2f4     pch.obj
 0002:000002f8       ?max_exponent@?$numeric_limits@N@std@@2HB 1000f2f8     pch.obj
 0002:000002fc       ?max_exponent10@?$numeric_limits@N@std@@2HB 1000f2fc     pch.obj
 0002:00000300       ?min_exponent@?$numeric_limits@N@std@@2HB 1000f300     pch.obj
 0002:00000304       ?min_exponent10@?$numeric_limits@N@std@@2HB 1000f304     pch.obj
 0002:00000308       ?digits@?$numeric_limits@O@std@@2HB 1000f308     pch.obj
 0002:0000030c       ?digits10@?$numeric_limits@O@std@@2HB 1000f30c     pch.obj
 0002:00000310       ?max_digits10@?$numeric_limits@O@std@@2HB 1000f310     pch.obj
 0002:00000314       ?max_exponent@?$numeric_limits@O@std@@2HB 1000f314     pch.obj
 0002:00000318       ?max_exponent10@?$numeric_limits@O@std@@2HB 1000f318     pch.obj
 0002:0000031c       ?min_exponent@?$numeric_limits@O@std@@2HB 1000f31c     pch.obj
 0002:00000320       ?min_exponent10@?$numeric_limits@O@std@@2HB 1000f320     pch.obj
 0002:00000324       ?value@?$integral_constant@H$0A@@std@@2HB 1000f324     pch.obj
 0002:00000328       ?has_denorm@_Num_base@std@@2W4float_denorm_style@2@B 1000f328     pch.obj
 0002:0000032c       ?has_denorm_loss@_Num_base@std@@2_NB 1000f32c     pch.obj
 0002:0000032d       ?has_infinity@_Num_base@std@@2_NB 1000f32d     pch.obj
 0002:0000032e       ?has_quiet_NaN@_Num_base@std@@2_NB 1000f32e     pch.obj
 0002:0000032f       ?has_signaling_NaN@_Num_base@std@@2_NB 1000f32f     pch.obj
 0002:00000330       ?is_bounded@_Num_base@std@@2_NB 1000f330     pch.obj
 0002:00000331       ?is_exact@_Num_base@std@@2_NB 1000f331     pch.obj
 0002:00000332       ?is_iec559@_Num_base@std@@2_NB 1000f332     pch.obj
 0002:00000333       ?is_integer@_Num_base@std@@2_NB 1000f333     pch.obj
 0002:00000334       ?is_modulo@_Num_base@std@@2_NB 1000f334     pch.obj
 0002:00000335       ?is_signed@_Num_base@std@@2_NB 1000f335     pch.obj
 0002:00000336       ?is_specialized@_Num_base@std@@2_NB 1000f336     pch.obj
 0002:00000337       ?tinyness_before@_Num_base@std@@2_NB 1000f337     pch.obj
 0002:00000338       ?traps@_Num_base@std@@2_NB 1000f338     pch.obj
 0002:0000033c       ?round_style@_Num_base@std@@2W4float_round_style@2@B 1000f33c     pch.obj
 0002:00000340       ?digits@_Num_base@std@@2HB 1000f340     pch.obj
 0002:00000344       ?digits10@_Num_base@std@@2HB 1000f344     pch.obj
 0002:00000348       ?max_digits10@_Num_base@std@@2HB 1000f348     pch.obj
 0002:0000034c       ?max_exponent@_Num_base@std@@2HB 1000f34c     pch.obj
 0002:00000350       ?max_exponent10@_Num_base@std@@2HB 1000f350     pch.obj
 0002:00000354       ?min_exponent@_Num_base@std@@2HB 1000f354     pch.obj
 0002:00000358       ?min_exponent10@_Num_base@std@@2HB 1000f358     pch.obj
 0002:0000035c       ?radix@_Num_base@std@@2HB  1000f35c     pch.obj
 0002:00000360       ?is_bounded@_Num_int_base@std@@2_NB 1000f360     pch.obj
 0002:00000361       ?is_exact@_Num_int_base@std@@2_NB 1000f361     pch.obj
 0002:00000362       ?is_integer@_Num_int_base@std@@2_NB 1000f362     pch.obj
 0002:00000363       ?is_modulo@_Num_int_base@std@@2_NB 1000f363     pch.obj
 0002:00000364       ?is_specialized@_Num_int_base@std@@2_NB 1000f364     pch.obj
 0002:00000368       ?radix@_Num_int_base@std@@2HB 1000f368     pch.obj
 0002:0000036c       ?value@?$_Sizeof@HU_Nil@std@@U12@U12@U12@U12@U12@U12@@std@@2IB 1000f36c     pch.obj
 0002:00000370       ?has_denorm@_Num_float_base@std@@2W4float_denorm_style@2@B 1000f370     pch.obj
 0002:00000374       ?has_denorm_loss@_Num_float_base@std@@2_NB 1000f374     pch.obj
 0002:00000375       ?has_infinity@_Num_float_base@std@@2_NB 1000f375     pch.obj
 0002:00000376       ?has_quiet_NaN@_Num_float_base@std@@2_NB 1000f376     pch.obj
 0002:00000377       ?has_signaling_NaN@_Num_float_base@std@@2_NB 1000f377     pch.obj
 0002:00000378       ?is_bounded@_Num_float_base@std@@2_NB 1000f378     pch.obj
 0002:00000379       ?is_exact@_Num_float_base@std@@2_NB 1000f379     pch.obj
 0002:0000037a       ?is_iec559@_Num_float_base@std@@2_NB 1000f37a     pch.obj
 0002:0000037b       ?is_integer@_Num_float_base@std@@2_NB 1000f37b     pch.obj
 0002:0000037c       ?is_modulo@_Num_float_base@std@@2_NB 1000f37c     pch.obj
 0002:0000037d       ?is_signed@_Num_float_base@std@@2_NB 1000f37d     pch.obj
 0002:0000037e       ?is_specialized@_Num_float_base@std@@2_NB 1000f37e     pch.obj
 0002:0000037f       ?tinyness_before@_Num_float_base@std@@2_NB 1000f37f     pch.obj
 0002:00000380       ?traps@_Num_float_base@std@@2_NB 1000f380     pch.obj
 0002:00000384       ?round_style@_Num_float_base@std@@2W4float_round_style@2@B 1000f384     pch.obj
 0002:00000388       ?radix@_Num_float_base@std@@2HB 1000f388     pch.obj
 0002:0000038c       ?is_signed@?$numeric_limits@D@std@@2_NB 1000f38c     pch.obj
 0002:00000390       ?digits@?$numeric_limits@D@std@@2HB 1000f390     pch.obj
 0002:00000394       ?digits10@?$numeric_limits@D@std@@2HB 1000f394     pch.obj
 0002:00000398       ?is_signed@?$numeric_limits@_W@std@@2_NB 1000f398     pch.obj
 0002:0000039c       ?digits@?$numeric_limits@_W@std@@2HB 1000f39c     pch.obj
 0002:000003a0       ?digits10@?$numeric_limits@_W@std@@2HB 1000f3a0     pch.obj
 0002:000003a4       ?is_modulo@?$numeric_limits@_N@std@@2_NB 1000f3a4     pch.obj
 0002:000003a5       ?is_signed@?$numeric_limits@_N@std@@2_NB 1000f3a5     pch.obj
 0002:000003a8       ?digits@?$numeric_limits@_N@std@@2HB 1000f3a8     pch.obj
 0002:000003ac       ?digits10@?$numeric_limits@_N@std@@2HB 1000f3ac     pch.obj
 0002:000003b0       ?is_signed@?$numeric_limits@C@std@@2_NB 1000f3b0     pch.obj
 0002:000003b4       ?digits@?$numeric_limits@C@std@@2HB 1000f3b4     pch.obj
 0002:000003b8       ?digits10@?$numeric_limits@C@std@@2HB 1000f3b8     pch.obj
 0002:000003c0       _lua_ident                 1000f3c0     lapi.obj
 0002:00000438       ??_C@_08JEIPHCP@no?5value?$AA@ 1000f438     lapi.obj
 0002:00000444       ??_C@_0CA@NGIABPA@invalid?5tag?5for?5a?5userdata?5?$CI?$CFd?$CJ?$AA@ 1000f444     lapi.obj
 0002:00000464       ??_C@_0BJ@COLEOPCM@reference?5table?5overflow?$AA@ 1000f464     lapi.obj
 0002:00000480       ??_C@_0CB@CKOJIFAK@cannot?5change?5the?5tag?5of?5a?5?$CF?420s@ 1000f480     lapi.obj
 0002:000004a4       ??_C@_01EFFIKLCJ@n?$AA@    1000f4a4     lapi.obj
 0002:000004a8       ??_C@_01OGPIMHDM@?$DP?$AA@ 1000f4a8     lauxlib.obj
 0002:000004ac       ??_C@_0CF@FEBLHFJI@bad?5argument?5?$CD?$CFd?5to?5?$GA?$CF?450s?8?5?$CI?$CF?41@ 1000f4ac     lauxlib.obj
 0002:000004d4       ??_C@_0BI@MKPNJCLI@?$CF?48s?5expected?0?5got?5?$CF?48s?$AA@ 1000f4d4     lauxlib.obj
 0002:000004ec       ??_C@_0BH@LBMGOGPM@stack?5overflow?5?$CI?$CF?430s?$CJ?$AA@ 1000f4ec     lauxlib.obj
 0002:00000504       ??_C@_0P@PDHEKNMA@value?5expected?$AA@ 1000f504     lauxlib.obj
 0002:00000518       __real@0000000000000000    1000f518     lauxlib.obj
 0002:00000520       ??_C@_06PDCMBPNP@_ALERT?$AA@ 1000f520     lbaselib.obj
 0002:00000528       ??_C@_08FNIIFOJC@tostring?$AA@ 1000f528     lbaselib.obj
 0002:00000678       ??_C@_02MFDMBIJM@ok?$AA@   1000f678     lbaselib.obj
 0002:0000067c       ??_C@_0P@EHLNGLLG@run?9time?5error?$AA@ 1000f67c     lbaselib.obj
 0002:0000068c       ??_C@_0L@KIJFAKBJ@file?5error?$AA@ 1000f68c     lbaselib.obj
 0002:00000698       ??_C@_0N@MNJHOOI@syntax?5error?$AA@ 1000f698     lbaselib.obj
 0002:000006a8       ??_C@_0N@FEGBBGML@memory?5error?$AA@ 1000f6a8     lbaselib.obj
 0002:000006b8       ??_C@_0BI@KGOCJOGJ@error?5in?5error?5handling?$AA@ 1000f6b8     lbaselib.obj
 0002:000006d0       ??_C@_0L@FKAAELBD@foreachvar?$AA@ 1000f6d0     lbaselib.obj
 0002:000006dc       ??_C@_07HHFJHNNN@nextvar?$AA@ 1000f6dc     lbaselib.obj
 0002:000006e4       ??_C@_0N@HICPLEMP@rawgetglobal?$AA@ 1000f6e4     lbaselib.obj
 0002:000006f4       ??_C@_0N@FGGKJFFN@rawsetglobal?$AA@ 1000f6f4     lbaselib.obj
 0002:00000704       ??_C@_05IJDJACGD@print?$AA@ 1000f704     lbaselib.obj
 0002:0000070c       ??_C@_08JOIMPOJO@tonumber?$AA@ 1000f70c     lbaselib.obj
 0002:00000718       ??_C@_04OMFAIDPG@call?$AA@ 1000f718     lbaselib.obj
 0002:00000720       ??_C@_0P@CKFEAJJE@collectgarbage?$AA@ 1000f720     lbaselib.obj
 0002:00000730       ??_C@_0P@GJPFIGAB@copytagmethods?$AA@ 1000f730     lbaselib.obj
 0002:00000740       ??_C@_06ONNDGCDK@dofile?$AA@ 1000f740     lbaselib.obj
 0002:00000748       ??_C@_08PBEIBMOD@dostring?$AA@ 1000f748     lbaselib.obj
 0002:00000754       ??_C@_05KKCIMGE@error?$AA@ 1000f754     lbaselib.obj
 0002:0000075c       ??_C@_07ICLAOFOB@foreach?$AA@ 1000f75c     lbaselib.obj
 0002:00000764       ??_C@_08GDLALCOF@foreachi?$AA@ 1000f764     lbaselib.obj
 0002:00000770       ??_C@_06EDAGHKOI@gcinfo?$AA@ 1000f770     lbaselib.obj
 0002:00000778       ??_C@_09CKJHDEOD@getglobal?$AA@ 1000f778     lbaselib.obj
 0002:00000784       ??_C@_04LGLBCCCL@getn?$AA@ 1000f784     lbaselib.obj
 0002:0000078c       ??_C@_0N@BBBHEOCE@gettagmethod?$AA@ 1000f78c     lbaselib.obj
 0002:0000079c       ??_C@_07NAPALOBA@globals?$AA@ 1000f79c     lbaselib.obj
 0002:000007a4       ??_C@_06CNCFNOLD@newtag?$AA@ 1000f7a4     lbaselib.obj
 0002:000007ac       ??_C@_04CJGEDOF@next?$AA@  1000f7ac     lbaselib.obj
 0002:000007b4       ??_C@_06DCIAHLCA@rawget?$AA@ 1000f7b4     lbaselib.obj
 0002:000007bc       ??_C@_06ONPLLLOI@rawset?$AA@ 1000f7bc     lbaselib.obj
 0002:000007c4       ??_C@_0M@INDDMEGM@rawgettable?$AA@ 1000f7c4     lbaselib.obj
 0002:000007d0       ??_C@_0M@HMBPNHBB@rawsettable?$AA@ 1000f7d0     lbaselib.obj
 0002:000007dc       ??_C@_09ENCBFHB@setglobal?$AA@ 1000f7dc     lbaselib.obj
 0002:000007e8       ??_C@_06GMIMFJGN@settag?$AA@ 1000f7e8     lbaselib.obj
 0002:000007f0       ??_C@_0N@GFKJICGI@settagmethod?$AA@ 1000f7f0     lbaselib.obj
 0002:00000800       ??_C@_03FJEPELFP@tag?$AA@  1000f800     lbaselib.obj
 0002:00000804       ??_C@_04GPMDFGEJ@type?$AA@ 1000f804     lbaselib.obj
 0002:0000080c       ??_C@_06OFCEDBEC@typeid?$AA@ 1000f80c     lbaselib.obj
 0002:00000814       ??_C@_06GMEIIFFN@assert?$AA@ 1000f814     lbaselib.obj
 0002:0000081c       ??_C@_04PIMMHFGE@sort?$AA@ 1000f81c     lbaselib.obj
 0002:00000824       ??_C@_07DALLEFAC@tinsert?$AA@ 1000f824     lbaselib.obj
 0002:0000082c       ??_C@_07NLBIDPLO@tremove?$AA@ 1000f82c     lbaselib.obj
 0002:00000834       ??_C@_0CL@EENDMONP@?$GAtostring?8?5must?5return?5a?5string?5@ 1000f834     lbaselib.obj
 0002:00000860       ??_C@_01GPOEFGEJ@?7?$AA@   1000f860     lbaselib.obj
 0002:00000864       ??_C@_0BC@GGLHLOMM@base?5out?5of?5range?$AA@ 1000f864     lbaselib.obj
 0002:00000878       ??_C@_0BJ@JFLPJELN@function?5or?5nil?5expected?$AA@ 1000f878     lbaselib.obj
 0002:00000894       ??_C@_02DPGMDCM@gc?$AA@    1000f894     lbaselib.obj
 0002:00000898       ??_C@_0DI@DELPBNIP@deprecated?5use?3?5cannot?5set?5the?5?$GA@ 1000f898     lbaselib.obj
 0002:000008d0       ??_C@_0DI@DGLOFNPB@deprecated?5use?3?5cannot?5get?5the?5?$GA@ 1000f8d0     lbaselib.obj
 0002:00000908       ??_C@_0CI@NKPNHOEJ@?$GAdostring?8?5cannot?5run?5pre?9compil@ 1000f908     lbaselib.obj
 0002:00000930       ??_C@_00CNPNBAHC@?$AA@     1000f930     lbaselib.obj
 0002:00000934       ??_C@_0O@LGIPBDLN@_ERRORMESSAGE?$AA@ 1000f934     lbaselib.obj
 0002:00000944       ??_C@_0BD@IOJAAODF@too?5many?5arguments?$AA@ 1000f944     lbaselib.obj
 0002:00000958       ??_C@_0CA@FLJBCEDH@deprecated?5option?5?$GAp?8?5in?5?$GAcall?8?$AA@ 1000f958     lbaselib.obj
 0002:00000978       ??_C@_09HEDEMKNG@table?3?5?$CFp?$AA@ 1000f978     lbaselib.obj
 0002:00000984       ??_C@_0N@KNPHMBNM@function?3?5?$CFp?$AA@ 1000f984     lbaselib.obj
 0002:00000994       ??_C@_0BB@KKIAPLCD@userdata?$CI?$CFd?$CJ?3?5?$CFp?$AA@ 1000f994     lbaselib.obj
 0002:000009a8       ??_C@_03ILAMHENH@nil?$AA@  1000f9a8     lbaselib.obj
 0002:000009ac       ??_C@_0BJ@PJKINODM@assertion?5failed?$CB?5?5?$CF?490s?$AA@ 1000f9ac     lbaselib.obj
 0002:000009c8       ??_C@_0CD@OFHMGIPD@invalid?5order?5function?5for?5sorti@ 1000f9c8     lbaselib.obj
 0002:000009ec       ??_C@_0BP@CDGMCKCO@function?5?$GA?$CF?420s?8?5is?5deprecated?$AA@ 1000f9ec     lbaselib.obj
 0002:00000a0c       ??_C@_07MKAKMJKM@Lua?54?40?$AA@ 1000fa0c     lbaselib.obj
 0002:00000a14       ??_C@_08PMLCGGEP@_VERSION?$AA@ 1000fa14     lbaselib.obj
 0002:00000a20       __real@4024000000000000    1000fa20     lbaselib.obj
 0002:00000a30       __xmm@41f00000000000000000000000000000 1000fa30     lbaselib.obj
 0002:00000aa0       _luaK_opproperties         1000faa0     lcode.obj
 0002:00000b34       ??_C@_0BL@BDOLDOFI@control?5structure?5too?5long?$AA@ 1000fb34     lcode.obj
 0002:00000b50       ??_C@_0CD@HGHHKJGL@function?5or?5expression?5too?5compl@ 1000fb50     lcode.obj
 0002:00000b74       ??_C@_0BI@DGLMJHJB@constant?5table?5overflow?$AA@ 1000fb74     lcode.obj
 0002:00000b8c       ??_C@_0BD@OHBABDDA@line?5info?5overflow?$AA@ 1000fb8c     lcode.obj
 0002:00000ba0       ??_C@_0BD@LKJEPOHE@code?5size?5overflow?$AA@ 1000fba0     lcode.obj
 0002:00000bb8       __real@417ffffff0000000    1000fbb8     lcode.obj
 0002:00000be8       ??_C@_08GMECKPDH@getlocal?$AA@ 1000fbe8     ldblib.obj
 0002:00000bf4       ??_C@_07OICKPAFH@getinfo?$AA@ 1000fbf4     ldblib.obj
 0002:00000bfc       ??_C@_0M@EMNFGEFA@setcallhook?$AA@ 1000fbfc     ldblib.obj
 0002:00000c08       ??_C@_0M@PABJPANF@setlinehook?$AA@ 1000fc08     ldblib.obj
 0002:00000c14       ??_C@_08JNGOLMEK@setlocal?$AA@ 1000fc14     ldblib.obj
 0002:00000c20       ??_C@_05CLBJLFDN@flnSu?$AA@ 1000fc20     ldblib.obj
 0002:00000c28       ??_C@_06NLLBKLAP@?$DO?$CF?410s?$AA@ 1000fc28     ldblib.obj
 0002:00000c30       ??_C@_0BL@NMONLLHA@function?5or?5level?5expected?$AA@ 1000fc30     ldblib.obj
 0002:00000c4c       ??_C@_0P@PJFAGLMH@invalid?5option?$AA@ 1000fc4c     ldblib.obj
 0002:00000c5c       ??_C@_06OEKOLKIL@source?$AA@ 1000fc5c     ldblib.obj
 0002:00000c64       ??_C@_09NOFDGFFO@short_src?$AA@ 1000fc64     ldblib.obj
 0002:00000c70       ??_C@_0M@IOFFDKM@linedefined?$AA@ 1000fc70     ldblib.obj
 0002:00000c7c       ??_C@_04IOPLPGDE@what?$AA@ 1000fc7c     ldblib.obj
 0002:00000c84       ??_C@_0M@OLGEEKJC@currentline?$AA@ 1000fc84     ldblib.obj
 0002:00000c90       ??_C@_04BDNNNDAF@nups?$AA@ 1000fc90     ldblib.obj
 0002:00000c98       ??_C@_04MEMAJGDJ@name?$AA@ 1000fc98     ldblib.obj
 0002:00000ca0       ??_C@_08JEGIFMFI@namewhat?$AA@ 1000fca0     ldblib.obj
 0002:00000cac       ??_C@_04HPNHAEOP@func?$AA@ 1000fcac     ldblib.obj
 0002:00000cb4       ??_C@_0BD@EFMIJNPC@level?5out?5of?5range?$AA@ 1000fcb4     ldblib.obj
 0002:00000cc8       ??_C@_0BC@GOAHAOGD@function?5expected?$AA@ 1000fcc8     ldblib.obj
 0002:00000cdc       ??_C@_03CBKFDHDL@Lua?$AA@  1000fcdc     ldebug.obj
 0002:00000ce0       ??_C@_0CK@IOFHDOLG@value?5for?5?$GAlua_getinfo?8?5is?5not?5a@ 1000fce0     ldebug.obj
 0002:00000d0c       ??_C@_02PHFJEMOI@?$DNC?$AA@ 1000fd0c     ldebug.obj
 0002:00000d10       ??_C@_01GFHCPBMG@C?$AA@    1000fd10     ldebug.obj
 0002:00000d14       ??_C@_04GHJNJNPO@main?$AA@ 1000fd14     ldebug.obj
 0002:00000d1c       ??_C@_06FJKEMHGD@global?$AA@ 1000fd1c     ldebug.obj
 0002:00000d24       ??_C@_0L@LMFFJDFH@tag?9method?$AA@ 1000fd24     ldebug.obj
 0002:00000d30       ??_C@_05IDKHKMLA@local?$AA@ 1000fd30     ldebug.obj
 0002:00000d38       ??_C@_05EIBGDMPB@field?$AA@ 1000fd38     ldebug.obj
 0002:00000d40       ??_C@_0CP@HGLPFCHJ@attempt?5to?5?$CF?430s?5?$CF?420s?5?$GA?$CF?440s?8?5?$CI@ 1000fd40     ldebug.obj
 0002:00000d70       ??_C@_0BP@DKJIDCM@attempt?5to?5?$CF?430s?5a?5?$CF?410s?5value?$AA@ 1000fd70     ldebug.obj
 0002:00000d90       ??_C@_0CE@IOFHEAFL@attempt?5to?5compare?5two?5?$CF?410s?5val@ 1000fd90     ldebug.obj
 0002:00000db4       ??_C@_0CE@HONJDMOC@attempt?5to?5compare?5?$CF?410s?5with?5?$CF?4@ 1000fdb4     ldebug.obj
 0002:00000dd8       ??_C@_0P@EODJGPIM@stack?5overflow?$AA@ 1000fdd8     ldo.obj
 0002:00000de8       ??_C@_04HJPCFDOP@line?$AA@ 1000fde8     ldo.obj
 0002:00000df0       ??_C@_06LNOFJDNM@return?$AA@ 1000fdf0     ldo.obj
 0002:00000df8       ??_C@_01KDCPPGHE@r?$AA@    1000fdf8     ldo.obj
 0002:00000dfc       ??_C@_02JDPG@rb?$AA@       1000fdfc     ldo.obj
 0002:00000e00       ??_C@_01EOFPKCAF@?$EA?$AA@ 1000fe00     ldo.obj
 0002:00000e04       ??_C@_07NBOOMMNB@?$CIstdin?$CJ?$AA@ 1000fe04     ldo.obj
 0002:00000e0c       ??_C@_0BM@IIIPLAIH@unable?5to?5recover?$DL?5exiting?6?$AA@ 1000fe0c     ldo.obj
 0002:00000ee8       ??_C@_03KCHOJKKI@set?$AA@  1000fee8     liolib.obj
 0002:00000eec       ??_C@_03LIBLMJMB@cur?$AA@  1000feec     liolib.obj
 0002:00000ef0       ??_C@_03JBJLGPFL@end?$AA@  1000fef0     liolib.obj
 0002:00000ef4       ??_C@_05DDECJJKE@clock?$AA@ 1000fef4     liolib.obj
 0002:00000efc       ??_C@_04JNIHBGGH@date?$AA@ 1000fefc     liolib.obj
 0002:00000f04       ??_C@_05GFCDIDHO@debug?$AA@ 1000ff04     liolib.obj
 0002:00000f0c       ??_C@_07EMGJIMLB@execute?$AA@ 1000ff0c     liolib.obj
 0002:00000f14       ??_C@_06EPDNLFGH@getenv?$AA@ 1000ff14     liolib.obj
 0002:00000f1c       ??_C@_06LEMKAMD@remove?$AA@ 1000ff1c     liolib.obj
 0002:00000f24       ??_C@_06LMEAOBLB@rename?$AA@ 1000ff24     liolib.obj
 0002:00000f2c       ??_C@_07KOJJABMD@tmpname?$AA@ 1000ff2c     liolib.obj
 0002:00000f34       ??_C@_08GJDELPHI@appendto?$AA@ 1000ff34     liolib.obj
 0002:00000f40       ??_C@_09BJJLCLMA@closefile?$AA@ 1000ff40     liolib.obj
 0002:00000f4c       ??_C@_05GLCAEPFP@flush?$AA@ 1000ff4c     liolib.obj
 0002:00000f54       ??_C@_08NEBHKOBO@openfile?$AA@ 1000ff54     liolib.obj
 0002:00000f60       ??_C@_04POLDLDMI@read?$AA@ 1000ff60     liolib.obj
 0002:00000f68       ??_C@_08KFJANHMN@readfrom?$AA@ 1000ff68     liolib.obj
 0002:00000f74       ??_C@_04EDECCOGL@seek?$AA@ 1000ff74     liolib.obj
 0002:00000f7c       ??_C@_05NGFEDHGN@write?$AA@ 1000ff7c     liolib.obj
 0002:00000f84       ??_C@_07NJHDNBFF@writeto?$AA@ 1000ff84     liolib.obj
 0002:00000f8c       ??_C@_06HDHHPPK@_INPUT?$AA@ 1000ff8c     liolib.obj
 0002:00000f94       ??_C@_07EKOFEPIK@_OUTPUT?$AA@ 1000ff94     liolib.obj
 0002:00000f9c       ??_C@_0BM@NHCEALGL@cannot?5access?5a?5closed?5file?$AA@ 1000ff9c     liolib.obj
 0002:00000fb8       ??_C@_0BE@BPELPPAA@invalid?5file?5handle?$AA@ 1000ffb8     liolib.obj
 0002:00000fcc       ??_C@_0CN@KENCKJFH@global?5variable?5?$GA?$CF?410s?8?5is?5not?5a@ 1000ffcc     liolib.obj
 0002:00000ffc       ??_C@_01NOFIACDB@w?$AA@    1000fffc     liolib.obj
 0002:00001000       ??_C@_01MCMALHOG@a?$AA@    10010000     liolib.obj
 0002:00001004       ??_C@_03DLDNIBIK@?$CFlf?$AA@ 10010004     liolib.obj
 0002:00001008       ??_C@_0CB@DOJBBJIC@not?5enough?5memory?5to?5read?5a?5file@ 10010008     liolib.obj
 0002:0000102c       ??_C@_02PMCMMBHA@?$CKl?$AA@ 1001002c     liolib.obj
 0002:00001030       ??_C@_0BN@ODDBPGME@read?5patterns?5are?5deprecated?$AA@ 10010030     liolib.obj
 0002:00001050       ??_C@_0P@CENJCLHM@invalid?5format?$AA@ 10010050     liolib.obj
 0002:00001060       ??_C@_05CFGAKADK@?$CF?416g?$AA@ 10010060     liolib.obj
 0002:00001068       ??_C@_0N@MICJCNHE@invalid?5mode?$AA@ 10010068     liolib.obj
 0002:00001078       ??_C@_02HAOIJKIC@?$CFc?$AA@ 10010078     liolib.obj
 0002:0000107c       ??_C@_0BG@LOLOKBOH@invalid?5?$GAdate?8?5format?$AA@ 1001007c     liolib.obj
 0002:00001094       ??_C@_0M@FBGICICO@lua_debug?$DO?5?$AA@ 10010094     liolib.obj
 0002:000010a0       ??_C@_05KJNBGLAC@cont?6?$AA@ 100100a0     liolib.obj
 0002:000010a8       ??_C@_0M@KGNBHMOP@parameter?3?5?$AA@ 100100a8     liolib.obj
 0002:000010b4       ??_C@_01EEMJAFIK@?6?$AA@   100100b4     liolib.obj
 0002:000010b8       ??_C@_0BC@GEKCAFLA@stack?5traceback?3?6?$AA@ 100100b8     liolib.obj
 0002:000010cc       ??_C@_0M@BAGMHIDI@?5?5?5?5?5?5?5?4?4?4?6?$AA@ 100100cc     liolib.obj
 0002:000010d8       ??_C@_06DOBANIAL@?$CF4d?3?5?5?$AA@ 100100d8     liolib.obj
 0002:000010e0       ??_C@_03IMACECCO@Snl?$AA@  100100e0     liolib.obj
 0002:000010e4       ??_C@_0BB@DMBKJKMH@function?5?$GA?$CF?450s?8?$AA@ 100100e4     liolib.obj
 0002:000010f8       ??_C@_0P@DGPABLPN@method?5?$GA?$CF?450s?8?$AA@ 100100f8     liolib.obj
 0002:00001108       ??_C@_0BD@CMLMEOGN@?$GA?$CF?450s?8?5tag?5method?$AA@ 10010108     liolib.obj
 0002:0000111c       ??_C@_0O@PEEGGO@main?5of?5?$CF?470s?$AA@ 1001011c     liolib.obj
 0002:0000112c       ??_C@_05CKCIFEAB@?$CF?470s?$AA@ 1001012c     liolib.obj
 0002:00001134       ??_C@_0BE@FLMFNC@function?5?$DM?$CFd?3?$CF?470s?$DO?$AA@ 10010134     liolib.obj
 0002:00001148       ??_C@_0M@BFHBKDJC@?5at?5line?5?$CFd?$AA@ 10010148     liolib.obj
 0002:00001154       ??_C@_08IJOAJNDI@?5?$FL?$CF?470s?$FN?$AA@ 10010154     liolib.obj
 0002:00001160       ??_C@_06PFEALBCD@_STDIN?$AA@ 10010160     liolib.obj
 0002:00001168       ??_C@_07EJFNLKNO@_STDOUT?$AA@ 10010168     liolib.obj
 0002:00001170       ??_C@_07HFPFOLLJ@_STDERR?$AA@ 10010170     liolib.obj
 0002:00001178       __real@408f400000000000    10010178     liolib.obj
 0002:000011f0       ??_C@_03BOPJPIAM@and?$AA@  100101f0     llex.obj
 0002:000011f4       ??_C@_05ELPHFHOI@break?$AA@ 100101f4     llex.obj
 0002:000011fc       ??_C@_02KNAFDCHJ@do?$AA@   100101fc     llex.obj
 0002:00001200       ??_C@_04FHMCPBIP@else?$AA@ 10010200     llex.obj
 0002:00001208       ??_C@_06CAACNEC@elseif?$AA@ 10010208     llex.obj
 0002:00001210       ??_C@_03JOHEBPFF@for?$AA@  10010210     llex.obj
 0002:00001214       ??_C@_08HFFPPCHF@function?$AA@ 10010214     llex.obj
 0002:00001220       ??_C@_02HEBPBKGD@if?$AA@   10010220     llex.obj
 0002:00001224       ??_C@_03NJKJADM@not?$AA@   10010224     llex.obj
 0002:00001228       ??_C@_02FODMLBIE@or?$AA@   10010228     llex.obj
 0002:0000122c       ??_C@_06LGDBIFHB@repeat?$AA@ 1001022c     llex.obj
 0002:00001234       ??_C@_04HOHPNOOD@then?$AA@ 10010234     llex.obj
 0002:0000123c       ??_C@_05FJMDOIMN@until?$AA@ 1001023c     llex.obj
 0002:00001244       ??_C@_05OODBEKIG@while?$AA@ 10010244     llex.obj
 0002:0000124c       ??_C@_02DJGKEECL@?4?4?$AA@ 1001024c     llex.obj
 0002:00001250       ??_C@_03KHICJKCI@?4?4?4?$AA@ 10010250     llex.obj
 0002:00001254       ??_C@_02EGOFBIJA@?$DN?$DN?$AA@ 10010254     llex.obj
 0002:00001258       ??_C@_02EEKDKGMJ@?$DO?$DN?$AA@ 10010258     llex.obj
 0002:0000125c       ??_C@_02EHCHHCKH@?$DM?$DN?$AA@ 1001025c     llex.obj
 0002:00001260       ??_C@_02DEDJCLAJ@?$HO?$DN?$AA@ 10010260     llex.obj
 0002:00001264       ??_C@_05CINCKAN@?$DMeof?$DO?$AA@ 10010264     llex.obj
 0002:0000126c       ??_C@_0BK@GLBMAEEH@too?5many?5?$CF?450s?5?$CIlimit?$DN?$CFd?$CJ?$AA@ 1001026c     llex.obj
 0002:00001288       ??_C@_0DG@LKDLDJA@?$CF?499s?$DL?6?5?5last?5token?5read?3?5?$GA?$CF?430s@ 10010288     llex.obj
 0002:000012c0       ??_C@_06IBAGLEAI@0x?$CF02X?$AA@ 100102c0     llex.obj
 0002:000012c8       ??_C@_0BF@EHKLJMMB@invalid?5control?5char?$AA@ 100102c8     llex.obj
 0002:000012e0       ??_C@_0BB@IGNCAHNA@lines?5in?5a?5chunk?$AA@ 100102e0     llex.obj
 0002:000012f4       ??_C@_0DI@KNOLHHPJ@ambiguous?5syntax?5?$CIdecimal?5point?5@ 100102f4     llex.obj
 0002:0000132c       ??_C@_0BB@CFMNENCE@malformed?5number?$AA@ 1001032c     llex.obj
 0002:00001340       ??_C@_0BH@BBMFLJJP@unfinished?5long?5string?$AA@ 10010340     llex.obj
 0002:00001358       ??_C@_0BC@IBAFBKML@unfinished?5string?$AA@ 10010358     llex.obj
 0002:0000136c       ??_C@_0BK@GLJFEJMO@escape?5sequence?5too?5large?$AA@ 1001036c     llex.obj
 0002:00001388       ??_C@_0DB@PPDGJHNG@unexpected?5?$GA$?8?5?$CIpragmas?5are?5no?5l@ 10010388     llex.obj
 0002:00001498       ??_C@_03BCGAIFPO@abs?$AA@  10010498     lmathlib.obj
 0002:0000149c       ??_C@_03BLEJJJBH@sin?$AA@  1001049c     lmathlib.obj
 0002:000014a0       ??_C@_03LALBNOCG@cos?$AA@  100104a0     lmathlib.obj
 0002:000014a4       ??_C@_03IIINPABG@tan?$AA@  100104a4     lmathlib.obj
 0002:000014a8       ??_C@_04FIHNOPOL@asin?$AA@ 100104a8     lmathlib.obj
 0002:000014b0       ??_C@_04PDIFKINK@acos?$AA@ 100104b0     lmathlib.obj
 0002:000014b8       ??_C@_04MLLJIGOK@atan?$AA@ 100104b8     lmathlib.obj
 0002:000014c0       ??_C@_05KNGEOGJB@atan2?$AA@ 100104c0     lmathlib.obj
 0002:000014c8       ??_C@_04GFPJNGEK@ceil?$AA@ 100104c8     lmathlib.obj
 0002:000014d0       ??_C@_05PBJFFIGL@floor?$AA@ 100104d0     lmathlib.obj
 0002:000014d8       ??_C@_03FFONCNID@mod?$AA@  100104d8     lmathlib.obj
 0002:000014dc       ??_C@_05GKKHEGJL@frexp?$AA@ 100104dc     lmathlib.obj
 0002:000014e4       ??_C@_05CEJMAHNP@ldexp?$AA@ 100104e4     lmathlib.obj
 0002:000014ec       ??_C@_04EIAKFFMI@sqrt?$AA@ 100104ec     lmathlib.obj
 0002:000014f4       ??_C@_03KLIPLJLL@min?$AA@  100104f4     lmathlib.obj
 0002:000014f8       ??_C@_03LJAEFNNE@max?$AA@  100104f8     lmathlib.obj
 0002:000014fc       ??_C@_03MGHMBJCF@log?$AA@  100104fc     lmathlib.obj
 0002:00001500       ??_C@_05HGHHAHAP@log10?$AA@ 10010500     lmathlib.obj
 0002:00001508       ??_C@_03KHJOGHMM@exp?$AA@  10010508     lmathlib.obj
 0002:0000150c       ??_C@_03OFPLEBM@deg?$AA@   1001050c     lmathlib.obj
 0002:00001510       ??_C@_03FHAJEHEA@rad?$AA@  10010510     lmathlib.obj
 0002:00001514       ??_C@_06NLFCANPD@random?$AA@ 10010514     lmathlib.obj
 0002:0000151c       ??_C@_0L@PIIACENG@randomseed?$AA@ 1001051c     lmathlib.obj
 0002:00001528       ??_C@_08COBKNEHN@math_and?$AA@ 10010528     lmathlib.obj
 0002:00001534       ??_C@_07IOPCJGL@math_or?$AA@ 10010534     lmathlib.obj
 0002:0000153c       ??_C@_08BIFOLNND@math_shl?$AA@ 1001053c     lmathlib.obj
 0002:00001548       ??_C@_08MMBPICAM@math_shr?$AA@ 10010548     lmathlib.obj
 0002:00001554       ??_C@_0BC@JKHEKPDC@interval?5is?5empty?$AA@ 10010554     lmathlib.obj
 0002:00001568       ??_C@_0BK@KNAOOCNO@wrong?5number?5of?5arguments?$AA@ 10010568     lmathlib.obj
 0002:00001584       ??_C@_03JGHBODFD@pow?$AA@  10010584     lmathlib.obj
 0002:00001588       ??_C@_02ENLJPMBB@PI?$AA@   10010588     lmathlib.obj
 0002:00001590       __real@3f91df46a2529d39    10010590     lmathlib.obj
 0002:00001598       __real@400921fb54442d18    10010598     lmathlib.obj
 0002:000015a0       __real@40dfffc000000000    100105a0     lmathlib.obj
 0002:000015a8       ??_C@_0CH@LBFPMMCP@memory?5allocation?5error?3?5block?5t@ 100105a8     lmem.obj
 0002:000015d0       _luaO_nilobject            100105d0     lobject.obj
 0002:000015e0       _luaO_typenames            100105e0     lobject.obj
 0002:000015f8       ??_C@_08NOEPOPLB@userdata?$AA@ 100105f8     lobject.obj
 0002:00001604       ??_C@_06EBGNBFIA@number?$AA@ 10010604     lobject.obj
 0002:0000160c       ??_C@_06ICGJLFIM@string?$AA@ 1001060c     lobject.obj
 0002:00001614       ??_C@_05LCLENNFI@table?$AA@ 10010614     lobject.obj
 0002:0000161c       ??_C@_0BA@EKNBFJDH@file?5?$GA?4?4?4?$CF?499s?8?$AA@ 1001061c     lobject.obj
 0002:0000162c       ??_C@_0N@NJDPHIHJ@file?5?$GA?$CF?499s?8?$AA@ 1001062c     lobject.obj
 0002:0000163c       ??_C@_08LDMCBCON@string?5?$CC?$AA@ 1001063c     lobject.obj
 0002:00001648       ??_C@_04JCKAGMEA@?4?4?4?$CC?$AA@ 10010648     lobject.obj
 0002:00001650       ??_C@_0P@NLJCCFPC@string?5?$CC?$CF?499s?$CC?$AA@ 10010650     lobject.obj
 0002:0000167c       ??_C@_0BB@BLJIODEI@?$GA?$CF?420s?8?5expected?$AA@ 1001067c     lparser.obj
 0002:00001690       ??_C@_0CP@KAIGMNJG@?$GA?$CF?420s?8?5expected?5?$CIto?5close?5?$GA?$CF?420@ 10010690     lparser.obj
 0002:000016c0       ??_C@_0BA@JPNMEOII@?$DMname?$DO?5expected?$AA@ 100106c0     lparser.obj
 0002:000016d0       ??_C@_0BA@EIDMAHJI@local?5variables?$AA@ 100106d0     lparser.obj
 0002:000016e0       ??_C@_0CI@OKCMGIOM@cannot?5access?5a?5variable?5in?5oute@ 100106e0     lparser.obj
 0002:00001708       ??_C@_08JKPCMKJ@upvalues?$AA@ 10010708     lparser.obj
 0002:00001714       ??_C@_0BO@DHCMJGEI@cannot?5access?5upvalue?5in?5main?$AA@ 10010714     lparser.obj
 0002:00001734       ??_C@_0DL@DENILDHB@upvalue?5must?5be?5global?5or?5local?5@ 10010734     lparser.obj
 0002:00001770       ??_C@_0L@HHPOFMCB@parameters?$AA@ 10010770     lparser.obj
 0002:0000177c       ??_C@_03CAOIPBNL@arg?$AA@  1001077c     lparser.obj
 0002:00001780       ??_C@_0P@NKPPCNBC@?$DMeof?$DO?5expected?$AA@ 10010780     lparser.obj
 0002:00001790       ??_C@_0BM@HEIHHEKF@function?5arguments?5expected?$AA@ 10010790     lparser.obj
 0002:000017ac       ??_C@_0BH@KMCCGJDG@?$DMname?$DO?5or?5?$GA?$FL?8?5expected?$AA@ 100107ac     lparser.obj
 0002:000017c4       ??_C@_0CE@LEIJHIGG@?$GAitem?5groups?8?5in?5a?5list?5initiali@ 100107c4     lparser.obj
 0002:000017e8       ??_C@_0BL@CBIHNBEM@invalid?5constructor?5syntax?$AA@ 100107e8     lparser.obj
 0002:00001804       ??_C@_0CA@CACCDEKA@elements?5in?5a?5table?5constructor?$AA@ 10010804     lparser.obj
 0002:00001824       ??_C@_0BG@KKIBCNLG@?$DMexpression?$DO?5expected?$AA@ 10010824     lparser.obj
 0002:0000183c       ??_C@_0CD@EPKLKKIF@variables?5in?5a?5multiple?5assignme@ 1001083c     lparser.obj
 0002:00001860       ??_C@_07ODJBHFGE@?$CIlimit?$CJ?$AA@ 10010860     lparser.obj
 0002:00001868       ??_C@_06DGKJOJA@?$CIstep?$CJ?$AA@ 10010868     lparser.obj
 0002:00001870       ??_C@_0O@KCDEGCAH@?$GAin?8?5expected?$AA@ 10010870     lparser.obj
 0002:00001880       ??_C@_02LMMGJAGL@in?$AA@   10010880     lparser.obj
 0002:00001884       ??_C@_07PDJJILAE@?$CItable?$CJ?$AA@ 10010884     lparser.obj
 0002:0000188c       ??_C@_0BE@MAHNHICJ@?$GA?$DN?8?5or?5?$GA?0?8?5expected?$AA@ 1001088c     lparser.obj
 0002:000018a0       ??_C@_0BB@DBFONGCK@no?5loop?5to?5break?$AA@ 100108a0     lparser.obj
 0002:000018b4       ??_C@_0BF@CIDJAB@?$DMstatement?$DO?5expected?$AA@ 100108b4     lparser.obj
 0002:000018cc       ??_C@_0BJ@JGHMPHBJ@?$DMname?$DO?5or?5?$GA?4?4?4?8?5expected?$AA@ 100108cc     lparser.obj
 0002:000018e8       ??_C@_04PJDNGLKJ@self?$AA@ 100108e8     lparser.obj
 0002:000018f0       ??_C@_0N@DJAMIFEP@?$CIno?5message?$CJ?$AA@ 100108f0     lstate.obj
 0002:00001900       ??_C@_0L@LELKNDMK@error?3?5?$CFs?6?$AA@ 10010900     lstate.obj
 0002:00001968       ??_C@_06GICABBBG@strlen?$AA@ 10010968     lstrlib.obj
 0002:00001970       ??_C@_06NAMJLKKD@strsub?$AA@ 10010970     lstrlib.obj
 0002:00001978       ??_C@_08ECJMOPAO@strlower?$AA@ 10010978     lstrlib.obj
 0002:00001984       ??_C@_08BJCCIELH@strupper?$AA@ 10010984     lstrlib.obj
 0002:00001990       ??_C@_07JCNDIGAF@strchar?$AA@ 10010990     lstrlib.obj
 0002:00001998       ??_C@_06MKHAOGF@strrep?$AA@ 10010998     lstrlib.obj
 0002:000019a0       ??_C@_05OJENGABA@ascii?$AA@ 100109a0     lstrlib.obj
 0002:000019a8       ??_C@_07FIHIHKEC@strbyte?$AA@ 100109a8     lstrlib.obj
 0002:000019b0       ??_C@_06DLEPGFEF@format?$AA@ 100109b0     lstrlib.obj
 0002:000019b8       ??_C@_07PFELJMPK@strfind?$AA@ 100109b8     lstrlib.obj
 0002:000019c0       ??_C@_04GOLEAPFD@gsub?$AA@ 100109c0     lstrlib.obj
 0002:000019c8       ??_C@_0N@FCPHIMMG@out?5of?5range?$AA@ 100109c8     lstrlib.obj
 0002:000019d8       ??_C@_0O@EAJJMEEM@invalid?5value?$AA@ 100109d8     lstrlib.obj
 0002:000019e8       ??_C@_0BG@LEHNKOGD@invalid?5capture?5index?$AA@ 100109e8     lstrlib.obj
 0002:00001a00       ??_C@_0BI@ECNPHIBF@invalid?5pattern?5capture?$AA@ 10010a00     lstrlib.obj
 0002:00001a18       ??_C@_0CC@HAKOPAIK@malformed?5pattern?5?$CIends?5with?5?$GA?$CF?8@ 10010a18     lstrlib.obj
 0002:00001a3c       ??_C@_0CA@MPLDKKDI@malformed?5pattern?5?$CImissing?5?$GA?$FN?8?$CJ?$AA@ 10010a3c     lstrlib.obj
 0002:00001a5c       ??_C@_0BD@NGJIMPLI@unbalanced?5pattern?$AA@ 10010a5c     lstrlib.obj
 0002:00001a70       ??_C@_0BC@IMEAEJPD@too?5many?5captures?$AA@ 10010a70     lstrlib.obj
 0002:00001a84       ??_C@_0BD@BFKNEALP@unfinished?5capture?$AA@ 10010a84     lstrlib.obj
 0002:00001a98       ??_C@_0L@NLFJOONJ@?$FO$?$CK?$CL?$DP?4?$CI?$FL?$CF?9?$AA@ 10010a98     lstrlib.obj
 0002:00001aa4       ??_C@_0BM@NDEBGBCF@string?5or?5function?5expected?$AA@ 10010aa4     lstrlib.obj
 0002:00001ac0       ??_C@_04MPDIABOK@?2000?$AA@ 10010ac0     lstrlib.obj
 0002:00001ac8       ??_C@_0BG@NEFIPCPG@?$FL?9?$CL?5?$CD0?$FN?$CK?$CI?$CFd?$CK?$CJ?$CF?4?$DP?$CI?$CFd?$CK?$CJ?$AA@ 10010ac8     lstrlib.obj
 0002:00001ae0       ??_C@_0CN@KALFEKPN@invalid?5format?5?$CIwidth?5or?5precisi@ 10010ae0     lstrlib.obj
 0002:00001b10       ??_C@_0BL@IFAEJJMF@invalid?5option?5in?5?$GAformat?8?$AA@ 10010b10     lstrlib.obj
 0002:00001b30       __real@3ff0000000000000    10010b30     lstrlib.obj
 0002:00001b38       __real@bff0000000000000    10010b38     lstrlib.obj
 0002:00001b40       ??_C@_0BD@BDIKLFBP@table?5index?5is?5nil?$AA@ 10010b40     ltable.obj
 0002:00001b54       ??_C@_0BH@EOHDEKEB@invalid?5key?5for?5?$GAnext?8?$AA@ 10010b54     ltable.obj
 0002:00001b6c       ??_C@_0P@KKABOKCO@table?5overflow?$AA@ 10010b6c     ltable.obj
 0002:00001b80       _luaT_eventname            10010b80     ltm.obj
 0002:00001c2c       ??_C@_08FNFBNONP@gettable?$AA@ 10010c2c     ltm.obj
 0002:00001c38       ??_C@_08KMHNMNKC@settable?$AA@ 10010c38     ltm.obj
 0002:00001c44       ??_C@_05FKHKFDID@index?$AA@ 10010c44     ltm.obj
 0002:00001c4c       ??_C@_03BDGOHNNK@add?$AA@  10010c4c     ltm.obj
 0002:00001c50       ??_C@_03KCMAIMAP@sub?$AA@  10010c50     ltm.obj
 0002:00001c54       ??_C@_03IMIFIBCN@mul?$AA@  10010c54     ltm.obj
 0002:00001c58       ??_C@_03FEJMGOGI@div?$AA@  10010c58     ltm.obj
 0002:00001c5c       ??_C@_03BAEAIDIN@unm?$AA@  10010c5c     ltm.obj
 0002:00001c60       ??_C@_02KCAKIFL@lt?$AA@    10010c60     ltm.obj
 0002:00001c64       ??_C@_06CMLIEHFC@concat?$AA@ 10010c64     ltm.obj
 0002:00001c6c       ??_C@_02FJPJILEL@le?$AA@   10010c6c     ltm.obj
 0002:00001c70       ??_C@_02GHFEHLK@gt?$AA@    10010c70     ltm.obj
 0002:00001c74       ??_C@_02FFKMGEKK@ge?$AA@   10010c74     ltm.obj
 0002:00001c78       ??_C@_0BM@DNKFKJF@event?5?$GA?$CF?450s?8?5is?5deprecated?$AA@ 10010c78     ltm.obj
 0002:00001c94       ??_C@_0CE@CMKCAFDB@event?5?$GAgc?8?5for?5tables?5is?5depreca@ 10010c94     ltm.obj
 0002:00001cb8       ??_C@_0CC@KONKBFJJ@?$GA?$CF?450s?8?5is?5not?5a?5valid?5event?5nam@ 10010cb8     ltm.obj
 0002:00001cdc       ??_C@_0BD@HKKNKCPL@tag?5table?5overflow?$AA@ 10010cdc     ltm.obj
 0002:00001cf0       ??_C@_0BG@MBLIJLPD@?$CFd?5is?5not?5a?5valid?5tag?$AA@ 10010cf0     ltm.obj
 0002:00001d08       ??_C@_0CD@EHPKIOAK@tag?5?$CFd?5was?5not?5created?5by?5?$GAnewta@ 10010d08     ltm.obj
 0002:00001d2c       ??_C@_0BC@GHCOCBB@?5with?5default?5tag?$AA@ 10010d2c     ltm.obj
 0002:00001d40       ??_C@_0DH@PENLBIOB@cannot?5change?5?$GA?$CF?420s?8?5tag?5method@ 10010d40     ltm.obj
 0002:00001d78       ??_C@_0CH@PNBCKDC@tag?5method?5must?5be?5a?5function?5?$CIo@ 10010d78     ltm.obj
 0002:00001da0       ??_C@_0CC@PJALPFOI@unexpected?5end?5of?5file?5in?5?$GA?$CF?499s@ 10010da0     lundump.obj
 0002:00001dc4       ??_C@_0BE@EIADBNAM@bad?5code?5in?5?$GA?$CF?499s?8?$AA@ 10010dc4     lundump.obj
 0002:00001dd8       ??_C@_0BJ@HBGEGMHL@bad?5signature?5in?5?$GA?$CF?499s?8?$AA@ 10010dd8     lundump.obj
 0002:00001df4       ??_C@_0DP@PFNKEJHG@virtual?5machine?5mismatch?5in?5?$GA?$CF?49@ 10010df4     lundump.obj
 0002:00001e34       ??_C@_0DO@NOPHDFIM@?$GA?$CF?499s?8?5too?5new?3?6?5?5read?5version?5@ 10010e34     lundump.obj
 0002:00001e74       ??_C@_0DP@EOLMAOED@?$GA?$CF?499s?8?5too?5old?3?6?5?5read?5version?5@ 10010e74     lundump.obj
 0002:00001eb4       ??_C@_0M@FJMPJFGL@sizeof?$CIint?$CJ?$AA@ 10010eb4     lundump.obj
 0002:00001ec0       ??_C@_0P@EIGKACCA@sizeof?$CIsize_t?$CJ?$AA@ 10010ec0     lundump.obj
 0002:00001ed0       ??_C@_0BE@NCADFBID@sizeof?$CIInstruction?$CJ?$AA@ 10010ed0     lundump.obj
 0002:00001ee4       ??_C@_0BB@FLBGLNIN@SIZE_INSTRUCTION?$AA@ 10010ee4     lundump.obj
 0002:00001ef8       ??_C@_07PPPCJAOM@SIZE_OP?$AA@ 10010ef8     lundump.obj
 0002:00001f00       ??_C@_06CDDPLDGA@SIZE_B?$AA@ 10010f00     lundump.obj
 0002:00001f08       ??_C@_0P@MBDEDIHC@sizeof?$CINumber?$CJ?$AA@ 10010f08     lundump.obj
 0002:00001f18       ??_C@_0DP@POCPBLIH@unknown?5number?5format?5in?5?$GA?$CF?499s?8@ 10010f18     lundump.obj
 0002:00001f58       ??_C@_0DA@HNGPJFFJ@?$GA?$CF?499s?8?5apparently?5contains?5more@ 10010f58     lundump.obj
 0002:00001f88       __real@41b2b9b0a15be612    10010f88     lundump.obj
 0002:00001f90       ??_C@_0BG@IOLALLOM@perform?5arithmetic?5on?$AA@ 10010f90     lvm.obj
 0002:00001fa8       ??_C@_0BF@IMDEEHDK@string?5size?5overflow?$AA@ 10010fa8     lvm.obj
 0002:00001fc0       ??_C@_0BE@CFOHABDI@undefined?5operation?$AA@ 10010fc0     lvm.obj
 0002:00001fd4       ??_C@_0BM@CPFDBJJK@?$GAfor?8?5step?5must?5be?5a?5number?$AA@ 10010fd4     lvm.obj
 0002:00001ff0       ??_C@_0BN@ODCLKLJN@?$GAfor?8?5limit?5must?5be?5a?5number?$AA@ 10010ff0     lvm.obj
 0002:00002010       ??_C@_0CF@POOBFDLI@?$GAfor?8?5initial?5value?5must?5be?5a?5nu@ 10011010     lvm.obj
 0002:00002038       ??_C@_0BN@JEAKHJPO@?$GAfor?8?5index?5must?5be?5a?5number?$AA@ 10011038     lvm.obj
 0002:00002058       ??_C@_0BM@CFNJMACO@?$GAfor?8?5table?5must?5be?5a?5table?$AA@ 10011058     lvm.obj
 0002:00002080       __xmm@80000000000000008000000000000000 10011080     lvm.obj
 0002:00002090       ??_C@_0P@BCPDJJEH@Mem?2LuaMem?4cpp?$AA@ 10011090     LuaMem.obj
 0002:000020a0       ??_C@_0BG@BMCGNFJB@Lua?5?9?9?5Critical?5error?$AA@ 100110a0     LuaMem.obj
 0002:000020b8       ___ascii_ctype             100110b8     Assist:AsciiCType.obj
 0002:00002138       ___ascii_ctype_space       10011138     Assist:AsciiCType.obj
 0002:0000213c       ___ascii_ctype_cntrl       1001113c     Assist:AsciiCType.obj
 0002:00002140       ___ascii_ctype_digit       10011140     Assist:AsciiCType.obj
 0002:00002144       ___ascii_ctype_digix       10011144     Assist:AsciiCType.obj
 0002:00002148       ___ascii_ctype_upper       10011148     Assist:AsciiCType.obj
 0002:0000214c       ___ascii_ctype_lower       1001114c     Assist:AsciiCType.obj
 0002:00002150       ___ascii_ctype_punct       10011150     Assist:AsciiCType.obj
 0002:00002154       ??_C@_07NEKHPBCG@English?$AA@ 10011154     Assist:AsciiCType.obj
 0002:0000215c       ?skipws@?$_Iosb@H@std@@2W4_Fmtflags@12@B 1001115c     Assist:pch.obj
 0002:00002160       ?unitbuf@?$_Iosb@H@std@@2W4_Fmtflags@12@B 10011160     Assist:pch.obj
 0002:00002164       ?uppercase@?$_Iosb@H@std@@2W4_Fmtflags@12@B 10011164     Assist:pch.obj
 0002:00002168       ?showbase@?$_Iosb@H@std@@2W4_Fmtflags@12@B 10011168     Assist:pch.obj
 0002:0000216c       ?showpoint@?$_Iosb@H@std@@2W4_Fmtflags@12@B 1001116c     Assist:pch.obj
 0002:00002170       ?showpos@?$_Iosb@H@std@@2W4_Fmtflags@12@B 10011170     Assist:pch.obj
 0002:00002174       ?left@?$_Iosb@H@std@@2W4_Fmtflags@12@B 10011174     Assist:pch.obj
 0002:00002178       ?right@?$_Iosb@H@std@@2W4_Fmtflags@12@B 10011178     Assist:pch.obj
 0002:0000217c       ?internal@?$_Iosb@H@std@@2W4_Fmtflags@12@B 1001117c     Assist:pch.obj
 0002:00002180       ?dec@?$_Iosb@H@std@@2W4_Fmtflags@12@B 10011180     Assist:pch.obj
 0002:00002184       ?oct@?$_Iosb@H@std@@2W4_Fmtflags@12@B 10011184     Assist:pch.obj
 0002:00002188       ?value@?$ice_and@$00$00$00$00$00$00$00@type_traits@boost@@2_NB 10011188     Assist:pch.obj
 0002:0000218c       ?hex@?$_Iosb@H@std@@2W4_Fmtflags@12@B 1001118c     Assist:pch.obj
 0002:00002190       ?scientific@?$_Iosb@H@std@@2W4_Fmtflags@12@B 10011190     Assist:pch.obj
 0002:00002194       ?fixed@?$_Iosb@H@std@@2W4_Fmtflags@12@B 10011194     Assist:pch.obj
 0002:00002198       ?hexfloat@?$_Iosb@H@std@@2W4_Fmtflags@12@B 10011198     Assist:pch.obj
 0002:0000219c       ?boolalpha@?$_Iosb@H@std@@2W4_Fmtflags@12@B 1001119c     Assist:pch.obj
 0002:000021a0       ?value@?$ice_not@$00@type_traits@boost@@2_NB 100111a0     Assist:pch.obj
 0002:000021a4       ?_Stdio@?$_Iosb@H@std@@2W4_Fmtflags@12@B 100111a4     Assist:pch.obj
 0002:000021a8       ?adjustfield@?$_Iosb@H@std@@2W4_Fmtflags@12@B 100111a8     Assist:pch.obj
 0002:000021ac       ?basefield@?$_Iosb@H@std@@2W4_Fmtflags@12@B 100111ac     Assist:pch.obj
 0002:000021b0       ?floatfield@?$_Iosb@H@std@@2W4_Fmtflags@12@B 100111b0     Assist:pch.obj
 0002:000021b4       ?goodbit@?$_Iosb@H@std@@2W4_Iostate@12@B 100111b4     Assist:pch.obj
 0002:000021b8       ?eofbit@?$_Iosb@H@std@@2W4_Iostate@12@B 100111b8     Assist:pch.obj
 0002:000021bc       ?failbit@?$_Iosb@H@std@@2W4_Iostate@12@B 100111bc     Assist:pch.obj
 0002:000021c0       ?badbit@?$_Iosb@H@std@@2W4_Iostate@12@B 100111c0     Assist:pch.obj
 0002:000021c4       ?_Hardfail@?$_Iosb@H@std@@2W4_Iostate@12@B 100111c4     Assist:pch.obj
 0002:000021c8       ?in@?$_Iosb@H@std@@2W4_Openmode@12@B 100111c8     Assist:pch.obj
 0002:000021cc       ?out@?$_Iosb@H@std@@2W4_Openmode@12@B 100111cc     Assist:pch.obj
 0002:000021d0       ?ate@?$_Iosb@H@std@@2W4_Openmode@12@B 100111d0     Assist:pch.obj
 0002:000021d4       ?app@?$_Iosb@H@std@@2W4_Openmode@12@B 100111d4     Assist:pch.obj
 0002:000021d8       ?trunc@?$_Iosb@H@std@@2W4_Openmode@12@B 100111d8     Assist:pch.obj
 0002:000021dc       ?_Nocreate@?$_Iosb@H@std@@2W4_Openmode@12@B 100111dc     Assist:pch.obj
 0002:000021e0       ?_Noreplace@?$_Iosb@H@std@@2W4_Openmode@12@B 100111e0     Assist:pch.obj
 0002:000021e4       ?binary@?$_Iosb@H@std@@2W4_Openmode@12@B 100111e4     Assist:pch.obj
 0002:000021e8       ?value@?$is_convertible_impl@XX@detail@boost@@2_NB 100111e8     Assist:pch.obj
 0002:000021ec       ?beg@?$_Iosb@H@std@@2W4_Seekdir@12@B 100111ec     Assist:pch.obj
 0002:000021f0       ?cur@?$_Iosb@H@std@@2W4_Seekdir@12@B 100111f0     Assist:pch.obj
 0002:000021f4       ?end@?$_Iosb@H@std@@2W4_Seekdir@12@B 100111f4     Assist:pch.obj
 0002:000021f8       ?value@?$is_convertible_impl@X$$CBX@detail@boost@@2_NB 100111f8     Assist:pch.obj
 0002:000021f9       ?value@?$is_convertible_impl@X$$CCX@detail@boost@@2_NB 100111f9     Assist:pch.obj
 0002:000021fa       ?value@?$is_convertible_impl@X$$CDX@detail@boost@@2_NB 100111fa     Assist:pch.obj
 0002:000021fc       ?_Stream_err@failure@ios_base@std@@0W4io_errc@43@B 100111fc     Assist:pch.obj
 0002:00002200       ?value@?$is_convertible_impl@$$CBXX@detail@boost@@2_NB 10011200     Assist:pch.obj
 0002:00002201       ?value@?$is_convertible_impl@$$CBX$$CBX@detail@boost@@2_NB 10011201     Assist:pch.obj
 0002:00002202       ?value@?$is_convertible_impl@$$CBX$$CCX@detail@boost@@2_NB 10011202     Assist:pch.obj
 0002:00002203       ?value@?$is_convertible_impl@$$CBX$$CDX@detail@boost@@2_NB 10011203     Assist:pch.obj
 0002:00002204       ?value@?$is_convertible_impl@$$CCXX@detail@boost@@2_NB 10011204     Assist:pch.obj
 0002:00002205       ?value@?$is_convertible_impl@$$CCX$$CBX@detail@boost@@2_NB 10011205     Assist:pch.obj
 0002:00002206       ?value@?$is_convertible_impl@$$CCX$$CCX@detail@boost@@2_NB 10011206     Assist:pch.obj
 0002:00002207       ?value@?$is_convertible_impl@$$CCX$$CDX@detail@boost@@2_NB 10011207     Assist:pch.obj
 0002:00002208       ?value@?$is_convertible_impl@$$CDXX@detail@boost@@2_NB 10011208     Assist:pch.obj
 0002:00002209       ?value@?$is_convertible_impl@$$CDX$$CBX@detail@boost@@2_NB 10011209     Assist:pch.obj
 0002:0000220a       ?value@?$is_convertible_impl@$$CDX$$CCX@detail@boost@@2_NB 1001120a     Assist:pch.obj
 0002:0000220b       ?value@?$is_convertible_impl@$$CDX$$CDX@detail@boost@@2_NB 1001120b     Assist:pch.obj
 0002:0000220c       ?collate@?$_Locbase@H@std@@2HB 1001120c     Assist:pch.obj
 0002:00002210       ?ctype@?$_Locbase@H@std@@2HB 10011210     Assist:pch.obj
 0002:00002214       ?monetary@?$_Locbase@H@std@@2HB 10011214     Assist:pch.obj
 0002:00002218       ?numeric@?$_Locbase@H@std@@2HB 10011218     Assist:pch.obj
 0002:0000221c       ?time@?$_Locbase@H@std@@2HB 1001121c     Assist:pch.obj
 0002:00002220       ?value@?$bool_@$0A@@mpl@boost@@2_NB 10011220     Assist:pch.obj
 0002:00002224       ?messages@?$_Locbase@H@std@@2HB 10011224     Assist:pch.obj
 0002:00002228       ?all@?$_Locbase@H@std@@2HB 10011228     Assist:pch.obj
 0002:0000222c       ?none@?$_Locbase@H@std@@2HB 1001122c     Assist:pch.obj
 0002:00002230       ?value@?$bool_@$00@mpl@boost@@2_NB 10011230     Assist:pch.obj
 0002:00002231       ?value@?$is_enum_impl@M@detail@boost@@2_NB 10011231     Assist:pch.obj
 0002:00002232       ?value@?$is_enum_impl@N@detail@boost@@2_NB 10011232     Assist:pch.obj
 0002:00002233       ?value@?$is_enum_impl@O@detail@boost@@2_NB 10011233     Assist:pch.obj
 0002:00002234       ?value@?$is_enum_impl@X@detail@boost@@2_NB 10011234     Assist:pch.obj
 0002:00002235       ?value@?$is_enum_impl@$$CBX@detail@boost@@2_NB 10011235     Assist:pch.obj
 0002:00002236       ?value@?$is_enum_impl@$$CCX@detail@boost@@2_NB 10011236     Assist:pch.obj
 0002:00002237       ?value@?$is_enum_impl@$$CDX@detail@boost@@2_NB 10011237     Assist:pch.obj
 0002:00002238       ?value@?$ice_or@$0A@$0A@$0A@$0A@$0A@$0A@$0A@@type_traits@boost@@2_NB 10011238     Assist:pch.obj
 0002:00002240       ??_7error_category@std@@6B@ 10011240     Assist:pch.obj
 0002:0000225c       ??_7_Generic_error_category@std@@6B@ 1001125c     Assist:pch.obj
 0002:00002274       ??_C@_07DCLBNMLN@generic?$AA@ 10011274     Assist:pch.obj
 0002:0000227c       ??_C@_0O@BFJCFAAK@unknown?5error?$AA@ 1001127c     Assist:pch.obj
 0002:00002290       ??_7_Iostream_error_category@std@@6B@ 10011290     Assist:pch.obj
 0002:000022a8       ??_C@_08LLGCOLLL@iostream?$AA@ 100112a8     Assist:pch.obj
 0002:000022b4       ??_C@_0BG@PADBLCHM@iostream?5stream?5error?$AA@ 100112b4     Assist:pch.obj
 0002:000022d0       ??_7_System_error_category@std@@6B@ 100112d0     Assist:pch.obj
 0002:000022e8       ??_C@_06FHFOAHML@system?$AA@ 100112e8     Assist:pch.obj
 0002:000022f0       ??_C@_0BI@CFPLBAOH@invalid?5string?5position?$AA@ 100112f0     Assist:pch.obj
 0002:00002308       ??_C@_0BA@JFNIOLAK@string?5too?5long?$AA@ 10011308     Assist:pch.obj
 0002:00002318       __pDefaultRawDllMain       10011318     MSVCRT:crtdll.obj
 0002:00002318       __pRawDllMain              10011318     MSVCRT:crtdll.obj
 0002:00002320       ??_7type_info@@6B@         10011320     MSVCRT:ti_inst.obj
 0002:00002324       ?ProcessDetach@NativeDll@<CrtImplementationDetails>@@0IB 10011324     MSVCRT:initsect.obj
 0002:00002328       ?ProcessAttach@NativeDll@<CrtImplementationDetails>@@0IB 10011328     MSVCRT:initsect.obj
 0002:0000232c       ?ThreadAttach@NativeDll@<CrtImplementationDetails>@@0IB 1001132c     MSVCRT:initsect.obj
 0002:00002330       ?ThreadDetach@NativeDll@<CrtImplementationDetails>@@0IB 10011330     MSVCRT:initsect.obj
 0002:00002334       ?ProcessVerifier@NativeDll@<CrtImplementationDetails>@@0IB 10011334     MSVCRT:initsect.obj
 0002:00002340       __load_config_used         10011340     MSVCRT:loadcfg.obj
 0002:000023f0       ??_R4error_category@std@@6B@ 100113f0     Assist:pch.obj
 0002:00002404       ??_R3error_category@std@@8 10011404     Assist:pch.obj
 0002:00002414       ??_R2error_category@std@@8 10011414     Assist:pch.obj
 0002:0000241c       ??_R1A@?0A@EA@error_category@std@@8 1001141c     Assist:pch.obj
 0002:00002438       ??_R4_Generic_error_category@std@@6B@ 10011438     Assist:pch.obj
 0002:0000244c       ??_R3_Generic_error_category@std@@8 1001144c     Assist:pch.obj
 0002:0000245c       ??_R2_Generic_error_category@std@@8 1001145c     Assist:pch.obj
 0002:00002468       ??_R1A@?0A@EA@_Generic_error_category@std@@8 10011468     Assist:pch.obj
 0002:00002484       ??_R4_Iostream_error_category@std@@6B@ 10011484     Assist:pch.obj
 0002:00002498       ??_R3_Iostream_error_category@std@@8 10011498     Assist:pch.obj
 0002:000024a8       ??_R2_Iostream_error_category@std@@8 100114a8     Assist:pch.obj
 0002:000024b8       ??_R1A@?0A@EA@_Iostream_error_category@std@@8 100114b8     Assist:pch.obj
 0002:000024d4       ??_R4_System_error_category@std@@6B@ 100114d4     Assist:pch.obj
 0002:000024e8       ??_R3_System_error_category@std@@8 100114e8     Assist:pch.obj
 0002:000024f8       ??_R2_System_error_category@std@@8 100114f8     Assist:pch.obj
 0002:00002508       ??_R1A@?0A@EA@_System_error_category@std@@8 10011508     Assist:pch.obj
 0002:00002524       ??_R4type_info@@6B@        10011524     MSVCRT:ti_inst.obj
 0002:00002538       ??_R3type_info@@8          10011538     MSVCRT:ti_inst.obj
 0002:00002548       ??_R2type_info@@8          10011548     MSVCRT:ti_inst.obj
 0002:00002550       ??_R1A@?0A@EA@type_info@@8 10011550     MSVCRT:ti_inst.obj
 0002:00002570       ___safe_se_handler_table   10011570     <linker-defined>
 0002:00002578       ___rtc_iaa                 10011578     MSVCRT:initsect.obj
 0002:0000257c       ___rtc_izz                 1001157c     MSVCRT:initsect.obj
 0002:00002580       ___rtc_taa                 10011580     MSVCRT:initsect.obj
 0002:00002584       ___rtc_tzz                 10011584     MSVCRT:initsect.obj
 0002:000026bc       __IMPORT_DESCRIPTOR_Debug  100116bc     Debug:Debug.dll
 0002:000026d0       __IMPORT_DESCRIPTOR_Memory 100116d0     Memory:Memory.dll
 0002:000026e4       __IMPORT_DESCRIPTOR_MSVCP110 100116e4     msvcprt:MSVCP110.dll
 0002:000026f8       __IMPORT_DESCRIPTOR_MSVCR110 100116f8     MSVCRT:MSVCR110.dll
 0002:0000270c       __IMPORT_DESCRIPTOR_KERNEL32 1001170c     kernel32:KERNEL32.dll
 0002:00002720       __NULL_IMPORT_DESCRIPTOR   10011720     Debug:Debug.dll
 0003:00000000       ?_Generic_object@?$_Error_objects@H@std@@2V_Generic_error_category@2@A 10013000     Assist:pch.obj
 0003:00000004       ?_Iostream_object@?$_Error_objects@H@std@@2V_Iostream_error_category@2@A 10013004     Assist:pch.obj
 0003:00000008       ?_System_object@?$_Error_objects@H@std@@2V_System_error_category@2@A 10013008     Assist:pch.obj
 0003:0000000c       ??_R0?AVerror_category@std@@@8 1001300c     Assist:pch.obj
 0003:00000030       ??_R0?AV_Generic_error_category@std@@@8 10013030     Assist:pch.obj
 0003:0000005c       ??_R0?AV_Iostream_error_category@std@@@8 1001305c     Assist:pch.obj
 0003:00000088       ??_R0?AV_System_error_category@std@@@8 10013088     Assist:pch.obj
 0003:000000c0       ??_R0?AVtype_info@@@8      100130c0     MSVCRT:ti_inst.obj
 0003:000000d8       ___isa_enabled             100130d8     MSVCRT:cpu_disp.obj
 0003:000000e0       ___native_dllmain_reason   100130e0     MSVCRT:natstart.obj
 0003:000000e4       ___security_cookie         100130e4     MSVCRT:gs_cookie.obj
 0003:000000e8       ___security_cookie_complement 100130e8     MSVCRT:gs_cookie.obj
 0003:00000100       ___@@_PchSym_@00@UsrxplibRkxhsrkUslnvdliowCxozhhrxUhixUrmgvinvwrzgvUulivrtmUofzUivovzhvUlyqUkxsOlyq@F96F8AB671AC0203 10013100     pch.obj
 0003:00000108       _g_outputCB                10013108     lbaselib.obj
 0003:0000010c       _g_alertCB                 1001310c     lbaselib.obj
 0003:00000120       ___@@_PchSym_@00@UsrxplibRkxhsrkUslnvdliowCxozhhrxUhixUrmgvinvwrzgvUhszivwUzhhrhgUivovzhvUlyqUkxsOlyq@7BF00F53649CB647 10013120     Assist:pch.obj
 0003:00000128       ?id@?$num_put@DV?$back_insert_iterator@V?$basic_string@DU?$char_traits@D@std@@V?$allocator@D@2@@std@@@std@@@std@@2V0locale@2@A 10013128     Assist:pch.obj
 0003:0000012c       ?id@?$num_put@_WV?$back_insert_iterator@V?$basic_string@_WU?$char_traits@_W@std@@V?$allocator@_W@2@@std@@@std@@@std@@2V0locale@2@A 1001312c     Assist:pch.obj
 0003:00000134       ___isa_available           10013134     MSVCRT:cpu_disp.obj
 0003:00000138       ___favor                   10013138     MSVCRT:cpu_disp.obj
 0003:0000013c       ?__type_info_root_node@@3U__type_info_node@@A 1001313c     MSVCRT:tncleanup.obj
 0003:00000480       _LUA_DBG_last_message      10013480     <common>
 0003:00000880       ___native_startup_lock     10013880     <common>
 0003:00000884       ___native_startup_state    10013884     <common>
 0003:00000888       ___dyn_tls_init_callback   10013888     <common>
 0003:0000088c       ___onexitend               1001388c     <common>
 0003:00000890       ___onexitbegin             10013890     <common>

 entry point at        0001:0000d096

 Static symbols

 0000:fffea000       .debug$S                   10000000     MSVCRT:MSVCR110.dll
 0000:fffea000       .debug$S                   10000000     MSVCRT:MSVCR110.dll
 0000:fffea000       .debug$S                   10000000     MSVCRT:MSVCR110.dll
 0000:fffea000       .debug$S                   10000000     MSVCRT:MSVCR110.dll
 0000:fffea000       .debug$S                   10000000     MSVCRT:MSVCR110.dll
 0000:fffea000       .debug$S                   10000000     MSVCRT:MSVCR110.dll
 0000:fffea000       .debug$S                   10000000     MSVCRT:MSVCR110.dll
 0000:fffea000       .debug$S                   10000000     MSVCRT:MSVCR110.dll
 0000:fffea000       .debug$S                   10000000     MSVCRT:MSVCR110.dll
 0000:fffea000       .debug$S                   10000000     MSVCRT:MSVCR110.dll
 0000:fffea000       .debug$S                   10000000     MSVCRT:MSVCR110.dll
 0000:fffea000       .debug$S                   10000000     MSVCRT:MSVCR110.dll
 0000:fffea000       .debug$S                   10000000     MSVCRT:MSVCR110.dll
 0000:fffea000       .debug$S                   10000000     MSVCRT:MSVCR110.dll
 0000:fffea000       .debug$S                   10000000     MSVCRT:MSVCR110.dll
 0000:fffea000       .debug$S                   10000000     MSVCRT:MSVCR110.dll
 0000:fffea000       .debug$S                   10000000     MSVCRT:MSVCR110.dll
 0000:fffea000       .debug$S                   10000000     MSVCRT:MSVCR110.dll
 0000:fffea000       .debug$S                   10000000     MSVCRT:MSVCR110.dll
 0000:fffea000       .debug$S                   10000000     MSVCRT:MSVCR110.dll
 0000:fffea000       .debug$S                   10000000     MSVCRT:MSVCR110.dll
 0000:fffea000       .debug$S                   10000000     MSVCRT:MSVCR110.dll
 0000:fffea000       .debug$S                   10000000     MSVCRT:MSVCR110.dll
 0000:fffea000       .debug$S                   10000000     MSVCRT:MSVCR110.dll
 0000:fffea000       .debug$S                   10000000     MSVCRT:MSVCR110.dll
 0000:fffea000       .debug$S                   10000000     MSVCRT:MSVCR110.dll
 0000:fffea000       .debug$S                   10000000     MSVCRT:MSVCR110.dll
 0000:fffea000       .debug$S                   10000000     MSVCRT:MSVCR110.dll
 0000:fffea000       .debug$S                   10000000     MSVCRT:MSVCR110.dll
 0000:fffea000       .debug$S                   10000000     MSVCRT:MSVCR110.dll
 0000:fffea000       .debug$S                   10000000     MSVCRT:MSVCR110.dll
 0000:fffea000       .debug$S                   10000000     MSVCRT:MSVCR110.dll
 0000:fffea000       .debug$S                   10000000     MSVCRT:MSVCR110.dll
 0000:fffea000       .debug$S                   10000000     MSVCRT:MSVCR110.dll
 0000:fffea000       .debug$S                   10000000     MSVCRT:MSVCR110.dll
 0000:fffea000       .debug$S                   10000000     MSVCRT:MSVCR110.dll
 0000:fffea000       .debug$S                   10000000     MSVCRT:MSVCR110.dll
 0000:fffea000       .debug$S                   10000000     MSVCRT:MSVCR110.dll
 0000:fffea000       .debug$S                   10000000     MSVCRT:MSVCR110.dll
 0000:fffea000       .debug$S                   10000000     MSVCRT:MSVCR110.dll
 0000:fffea000       .debug$S                   10000000     MSVCRT:MSVCR110.dll
 0000:fffea000       .debug$S                   10000000     MSVCRT:MSVCR110.dll
 0000:fffea000       .debug$S                   10000000     MSVCRT:MSVCR110.dll
 0000:fffea000       .debug$S                   10000000     MSVCRT:MSVCR110.dll
 0000:fffea000       .debug$S                   10000000     MSVCRT:MSVCR110.dll
 0000:fffea000       .debug$S                   10000000     MSVCRT:MSVCR110.dll
 0000:fffea000       .debug$S                   10000000     MSVCRT:MSVCR110.dll
 0000:fffea000       .debug$S                   10000000     MSVCRT:MSVCR110.dll
 0000:fffea000       .debug$S                   10000000     MSVCRT:MSVCR110.dll
 0000:fffea000       .debug$S                   10000000     MSVCRT:MSVCR110.dll
 0000:fffea000       .debug$S                   10000000     MSVCRT:MSVCR110.dll
 0000:fffea000       .debug$S                   10000000     MSVCRT:MSVCR110.dll
 0000:fffea000       .debug$S                   10000000     MSVCRT:MSVCR110.dll
 0000:fffea000       .debug$S                   10000000     MSVCRT:MSVCR110.dll
 0000:fffea000       .debug$S                   10000000     MSVCRT:MSVCR110.dll
 0000:fffea000       .debug$S                   10000000     MSVCRT:MSVCR110.dll
 0000:fffea000       .debug$S                   10000000     MSVCRT:MSVCR110.dll
 0000:fffea000       .debug$S                   10000000     MSVCRT:MSVCR110.dll
 0000:fffea000       .debug$S                   10000000     MSVCRT:MSVCR110.dll
 0000:fffea000       .debug$S                   10000000     MSVCRT:MSVCR110.dll
 0000:fffea000       .debug$S                   10000000     MSVCRT:MSVCR110.dll
 0000:fffea000       .debug$S                   10000000     MSVCRT:MSVCR110.dll
 0000:fffea000       .debug$S                   10000000     MSVCRT:MSVCR110.dll
 0000:fffea000       .debug$S                   10000000     MSVCRT:MSVCR110.dll
 0000:fffea000       .debug$S                   10000000     MSVCRT:MSVCR110.dll
 0000:fffea000       .debug$S                   10000000     MSVCRT:MSVCR110.dll
 0000:fffea000       .debug$S                   10000000     MSVCRT:MSVCR110.dll
 0000:fffea000       .debug$S                   10000000     MSVCRT:MSVCR110.dll
 0000:fffea000       .debug$S                   10000000     MSVCRT:MSVCR110.dll
 0000:fffea000       .debug$S                   10000000     MSVCRT:MSVCR110.dll
 0000:fffea000       .debug$S                   10000000     MSVCRT:MSVCR110.dll
 0000:fffea000       .debug$S                   10000000     MSVCRT:MSVCR110.dll
 0000:fffea000       .debug$S                   10000000     MSVCRT:MSVCR110.dll
 0000:fffea000       .debug$S                   10000000     MSVCRT:MSVCR110.dll
 0000:fffea000       .debug$S                   10000000     MSVCRT:MSVCR110.dll
 0000:fffea000       .debug$S                   10000000     MSVCRT:MSVCR110.dll
 0000:fffea000       .debug$S                   10000000     MSVCRT:MSVCR110.dll
 0000:fffea000       .debug$S                   10000000     MSVCRT:MSVCR110.dll
 0000:fffea000       .debug$S                   10000000     MSVCRT:MSVCR110.dll
 0000:fffea000       .debug$S                   10000000     MSVCRT:MSVCR110.dll
 0000:fffea000       .debug$S                   10000000     MSVCRT:MSVCR110.dll
 0000:fffea000       .debug$S                   10000000     MSVCRT:MSVCR110.dll
 0000:fffea000       .debug$S                   10000000     MSVCRT:MSVCR110.dll
 0000:fffea000       .debug$S                   10000000     MSVCRT:MSVCR110.dll
 0000:fffea000       .debug$S                   10000000     MSVCRT:MSVCR110.dll
 0000:fffea000       .debug$S                   10000000     MSVCRT:MSVCR110.dll
 0000:fffea000       .debug$S                   10000000     MSVCRT:MSVCR110.dll
 0000:fffea000       .debug$S                   10000000     MSVCRT:MSVCR110.dll
 0000:fffea000       .debug$S                   10000000     MSVCRT:MSVCR110.dll
 0000:fffea000       .debug$S                   10000000     MSVCRT:MSVCR110.dll
 0000:fffea000       .debug$S                   10000000     MSVCRT:MSVCR110.dll
 0000:fffea000       .debug$S                   10000000     MSVCRT:MSVCR110.dll
 0000:fffea000       .debug$S                   10000000     MSVCRT:MSVCR110.dll
 0000:fffea000       .debug$S                   10000000     msvcprt:MSVCP110.dll
 0000:fffea000       .debug$S                   10000000     msvcprt:MSVCP110.dll
 0000:fffea000       .debug$S                   10000000     msvcprt:MSVCP110.dll
 0000:fffea000       .debug$S                   10000000     msvcprt:MSVCP110.dll
 0000:fffea000       .debug$S                   10000000     msvcprt:MSVCP110.dll
 0000:fffea000       .debug$S                   10000000     msvcprt:MSVCP110.dll
 0000:fffea000       .debug$S                   10000000     Memory:Memory.dll
 0000:fffea000       .debug$S                   10000000     Memory:Memory.dll
 0000:fffea000       .debug$S                   10000000     Memory:Memory.dll
 0000:fffea000       .debug$S                   10000000     Memory:Memory.dll
 0000:fffea000       .debug$S                   10000000     Debug:Debug.dll
 0000:fffea000       .debug$S                   10000000     Debug:Debug.dll
 0000:fffea000       .debug$S                   10000000     Debug:Debug.dll
 0000:fffea000       .debug$S                   10000000     kernel32:KERNEL32.dll
 0000:fffea000       .debug$S                   10000000     kernel32:KERNEL32.dll
 0000:fffea000       .debug$S                   10000000     kernel32:KERNEL32.dll
 0000:fffea000       .debug$S                   10000000     kernel32:KERNEL32.dll
 0000:fffea000       .debug$S                   10000000     kernel32:KERNEL32.dll
 0000:fffea000       .debug$S                   10000000     kernel32:KERNEL32.dll
 0000:fffea000       .debug$S                   10000000     kernel32:KERNEL32.dll
 0000:fffea000       .debug$S                   10000000     kernel32:KERNEL32.dll
 0000:fffea000       .debug$S                   10000000     kernel32:KERNEL32.dll
 0001:0000002a       _luaA_indexAcceptable@8    1000102a f   lapi.obj
 0001:00000a07       _adjuststack@4             10001a07 f   lauxlib.obj
 0001:00000a7c       _emptybuffer@4             10001a7c f   lauxlib.obj
 0001:00000e17       _type_error@12             10001e17 f   lauxlib.obj
 0001:00000e63       _luaB__ALERT@4             10001e63 f   lbaselib.obj
 0001:00000e85       _luaB_print@4              10001e85 f   lbaselib.obj
 0001:00000f0e       _luaB_tonumber@4           10001f0e f   lbaselib.obj
 0001:00000ffc       _luaB_error@4              10001ffc f   lbaselib.obj
 0001:0000101a       _luaB_setglobal@4          1000201a f   lbaselib.obj
 0001:00001041       _luaB_getglobal@4          10002041 f   lbaselib.obj
 0001:0000105e       _luaB_tag@4                1000205e f   lbaselib.obj
 0001:00001092       _luaB_settag@4             10002092 f   lbaselib.obj
 0001:000010ca       _luaB_newtag@4             100020ca f   lbaselib.obj
 0001:000010f1       _luaB_copytagmethods@4     100020f1 f   lbaselib.obj
 0001:0000113a       _luaB_globals@4            1000213a f   lbaselib.obj
 0001:00001171       _luaB_rawget@4             10002171 f   lbaselib.obj
 0001:0000119a       _luaB_rawset@4             1000219a f   lbaselib.obj
 0001:000011ce       _luaB_settagmethod@4       100021ce f   lbaselib.obj
 0001:0000125a       _luaB_gettagmethod@4       1000225a f   lbaselib.obj
 0001:000012b2       _luaB_gcinfo@4             100022b2 f   lbaselib.obj
 0001:000012fa       _luaB_collectgarbage@4     100022fa f   lbaselib.obj
 0001:00001323       _luaB_type@4               10002323 f   lbaselib.obj
 0001:00001353       _luaB_typeid@4             10002353 f   lbaselib.obj
 0001:0000137c       _luaB_next@4               1000237c f   lbaselib.obj
 0001:000013b7       _luaB_dostring@4           100023b7 f   lbaselib.obj
 0001:0000140b       _luaB_dofile@4             1000240b f   lbaselib.obj
 0001:0000143f       _luaB_call@4               1000243f f   lbaselib.obj
 0001:0000155a       _luaB_tostring@4           1000255a f   lbaselib.obj
 0001:00001609       _luaB_foreachi@4           10002609 f   lbaselib.obj
 0001:0000168a       _luaB_foreach@4            1000268a f   lbaselib.obj
 0001:000016f7       _luaB_assert@4             100026f7 f   lbaselib.obj
 0001:0000173b       _luaB_getn@4               1000273b f   lbaselib.obj
 0001:00001771       _luaB_tinsert@4            10002771 f   lbaselib.obj
 0001:00001815       _luaB_tremove@4            10002815 f   lbaselib.obj
 0001:000018ca       _luaB_sort@4               100028ca f   lbaselib.obj
 0001:00001913       _auxsort@12                10002913 f   lbaselib.obj
 0001:00001b08       _deprecated_func@4         10002b08 f   lbaselib.obj
 0001:00001b2a       _deprecated_funcs@4        10002b2a f   lbaselib.obj
 0001:00001be6       _passresults@12            10002be6 f   lbaselib.obj
 0001:00001c2b       _set2@12                   10002c2b f   lbaselib.obj
 0001:00001c64       _sort_comp@12              10002c64 f   lbaselib.obj
 0001:00001cd2       _code_label@12             10002cd2 f   lcode.obj
 0001:00001ce0       _codelineinfo@4            10002ce0 f   lcode.obj
 0001:00001d4b       _discharge1@8              10002d4b f   lcode.obj
 0001:00001d75       _discharge@8               10002d75 f   lcode.obj
 0001:00001dc3       _invertjump@4              10002dc3 f   lcode.obj
 0001:00001dff       $LN16                      10002dff     lcode.obj
 0001:0000223f       _luaK_fixjump@12           1000323f f   lcode.obj
 0001:000022a3       _luaK_getjump@8            100032a3 f   lcode.obj
 0001:000022f2       _luaK_goiffalse@12         100032f2 f   lcode.obj
 0001:0000245a       _luaK_patchlistaux@20      1000345a f   lcode.obj
 0001:0000263b       _luaK_testgo@16            1000363b f   lcode.obj
 0001:00002801       _need_value@12             10003801 f   lcode.obj
 0001:0000283b       _number_constant@12        1000383b f   lcode.obj
 0001:000028b5       _previous_instruction@4    100038b5 f   lcode.obj
 0001:000028d1       _getinfo@4                 100038d1 f   ldblib.obj
 0001:00002a41       _getlocal@4                10003a41 f   ldblib.obj
 0001:00002ab2       _setlocal@4                10003ab2 f   ldblib.obj
 0001:00002b14       _setcallhook@4             10003b14 f   ldblib.obj
 0001:00002b32       _setlinehook@4             10003b32 f   ldblib.obj
 0001:00002b50       _callf@8                   10003b50 f   ldblib.obj
 0001:00002b70       _hookf@8                   10003b70 f   ldblib.obj
 0001:00002bc6       _linef@8                   10003bc6 f   ldblib.obj
 0001:00002c07       _sethook@16                10003c07 f   ldblib.obj
 0001:00002c89       _settabsi@12               10003c89 f   ldblib.obj
 0001:00002cbd       _settabss@12               10003cbd f   ldblib.obj
 0001:00002ce4       _aux_stackedfunction@12    10003ce4 f   ldebug.obj
 0001:00002d24       _currentline@4             10003d24 f   ldebug.obj
 0001:00002d57       _currentpc@4               10003d57 f   ldebug.obj
 0001:00002d7a       _funcinfo@12               10003d7a f   ldebug.obj
 0001:00002e01       _getfuncname@12            10003e01 f   ldebug.obj
 0001:00002e63       _getluaproto@4             10003e63 f   ldebug.obj
 0001:00002e7f       _getname@12                10003e7f f   ldebug.obj
 0001:00002f4c       _getobjname@12             10003f4c f   ldebug.obj
 0001:00002fe4       _infoLproto@8              10003fe4 f   ldebug.obj
 0001:00003005       _isLmark@4                 10004005 f   ldebug.obj
 0001:000030ff       _luaG_symbexec@12          100040ff f   ldebug.obj
 0001:0000349c       _nups@4                    1000449c f   ldebug.obj
 0001:000034bf       _pushpc@16                 100044bf f   ldebug.obj
 0001:000034e5       _setnormalized@8           100044e5 f   ldebug.obj
 0001:00003511       _travglobals@8             10004511 f   ldebug.obj
 0001:0000355e       _travtagmethods@8          1000455e f   ldebug.obj
 0001:000035a4       _callCclosure@12           100045a4 f   ldo.obj
 0001:00003602       _dohook@12                 10004602 f   ldo.obj
 0001:00003638       _f_call@8                  10004638 f   ldo.obj
 0001:0000364d       _f_parser@8                1000464d f   ldo.obj
 0001:00003817       _luaD_callHook@16          10004817 f   ldo.obj
 0001:00003932       _luaD_openstack@8          10004932 f   ldo.obj
 0001:00003aed       _message@8                 10004aed f   ldo.obj
 0001:00003b5a       _parse_buffer@16           10004b5a f   ldo.obj
 0001:00003ba2       _parse_file@8              10004ba2 f   ldo.obj
 0001:00003c9d       _protectedparser@12        10004c9d f   ldo.obj
 0001:00003ce8       _restore_stack_limit@4     10004ce8 f   ldo.obj
 0001:00003e85       _protosize@4               10004e85 f   lfunc.obj
 0001:00003eab       _callgcTM@8                10004eab f   lgc.obj
 0001:00003f10       _callgcTMudata@4           10004f10 f   lgc.obj
 0001:00003f72       _checkMbuffer@4            10004f72 f   lgc.obj
 0001:00003fa1       _checktab@8                10004fa1 f   lgc.obj
 0001:00003fcf       _collectclosure@4          10004fcf f   lgc.obj
 0001:00003ffe       _collectproto@4            10004ffe f   lgc.obj
 0001:00004032       _collectstrings@8          10005032 f   lgc.obj
 0001:0000409c       _collecttable@4            1000509c f   lgc.obj
 0001:000040cb       _collectudata@8            100050cb f   lgc.obj
 0001:0000413c       _hasmark@4                 1000513c f   lgc.obj
 0001:00004177       _invalidaterefs@4          10005177 f   lgc.obj
 0001:00004387       _luaC_collectgarbage@4     10005387 f   lgc.obj
 0001:0000442f       _markall@4                 1000542f f   lgc.obj
 0001:00004551       _markclosure@8             10005551 f   lgc.obj
 0001:0000457a       _marklock@8                1000557a f   lgc.obj
 0001:000045ae       _markobject@8              100055ae f   lgc.obj
 0001:00004609       _markstack@8               10005609 f   lgc.obj
 0001:0000462a       _marktagmethods@8          1000562a f   lgc.obj
 0001:0000466a       _protomark@4               1000566a f   lgc.obj
 0001:000046e6       _io_read@4                 100056e6 f   liolib.obj
 0001:00004855       _io_write@4                10005855 f   liolib.obj
 0001:0000491a       _io_seek@4                 1000591a f   liolib.obj
 0001:000049d2       _io_flush@4                100059d2 f   liolib.obj
 0001:00004a2c       _io_execute@4              10005a2c f   liolib.obj
 0001:00004a5d       _io_remove@4               10005a5d f   liolib.obj
 0001:00004a84       _io_rename@4               10005a84 f   liolib.obj
 0001:00004aba       _io_tmpname@4              10005aba f   liolib.obj
 0001:00004ad3       _io_getenv@4               10005ad3 f   liolib.obj
 0001:00004af8       _io_clock@4                10005af8 f   liolib.obj
 0001:00004b24       _io_date@4                 10005b24 f   liolib.obj
 0001:00004b96       _io_debug@4                10005b96 f   liolib.obj
 0001:00004ea9       _io_close@4                10005ea9 f   liolib.obj
 0001:00004ede       _io_open@4                 10005ede f   liolib.obj
 0001:00004f34       _io_readfrom@4             10005f34 f   liolib.obj
 0001:00004f47       _io_writeto@4              10005f47 f   liolib.obj
 0001:00004f5a       _io_appendto@4             10005f5a f   liolib.obj
 0001:00004f9f       _closefile@12              10005f9f f   liolib.obj
 0001:00004ff7       _file_collect@4            10005ff7 f   liolib.obj
 0001:0000503f       _getfilebyref@12           1000603f f   liolib.obj
 0001:00005091       _gethandle@12              10006091 f   liolib.obj
 0001:000050d6       _getnonullfile@12          100060d6 f   liolib.obj
 0001:00005105       _io_fromto@12              10006105 f   liolib.obj
 0001:00005197       _localtime                 10006197 f   liolib.obj
 0001:000051c5       _openwithcontrol@4         100061c5 f   liolib.obj
 0001:000052be       _pushresult@8              100062be f   liolib.obj
 0001:0000531c       _read_chars@12             1000631c f   liolib.obj
 0001:000053a7       _read_file@8               100063a7 f   liolib.obj
 0001:00005411       _read_line@8               10006411 f   liolib.obj
 0001:0000549d       _read_number@8             1000649d f   liolib.obj
 0001:000054db       _read_word@8               100064db f   liolib.obj
 0001:0000559a       _setfilebyname@16          1000659a f   liolib.obj
 0001:000055bd       _setreturn@16              100065bd f   liolib.obj
 0001:00005602       _time                      10006602 f   liolib.obj
 0001:00005608       _inclinenumber@4           10006608 f   llex.obj
 0001:000056e9       _luaX_invalidchar@8        100066e9 f   llex.obj
 0001:00005cd2       _read_long_string@8        10006cd2 f   llex.obj
 0001:00005ea5       _read_number@12            10006ea5 f   llex.obj
 0001:000060e8       _read_string@12            100070e8 f   llex.obj
 0001:00006388       _readname@4                10007388 f   llex.obj
 0001:00006424       _math_and@4                10007424 f   lmathlib.obj
 0001:0000646f       _math_or@4                 1000746f f   lmathlib.obj
 0001:000064ba       _math_shl@4                100074ba f   lmathlib.obj
 0001:00006505       _math_shr@4                10007505 f   lmathlib.obj
 0001:00006550       _math_abs@4                10007550 f   lmathlib.obj
 0001:00006577       _math_sin@4                10007577 f   lmathlib.obj
 0001:000065b4       _math_cos@4                100075b4 f   lmathlib.obj
 0001:000065f1       _math_tan@4                100075f1 f   lmathlib.obj
 0001:0000662e       _math_asin@4               1000762e f   lmathlib.obj
 0001:0000666b       _math_acos@4               1000766b f   lmathlib.obj
 0001:000066a8       _math_atan@4               100076a8 f   lmathlib.obj
 0001:000066e5       _math_atan2@4              100076e5 f   lmathlib.obj
 0001:00006734       _math_ceil@4               10007734 f   lmathlib.obj
 0001:0000675c       _math_floor@4              1000775c f   lmathlib.obj
 0001:00006784       _math_mod@4                10007784 f   lmathlib.obj
 0001:000067bd       _math_sqrt@4               100077bd f   lmathlib.obj
 0001:000067e4       _math_log@4                100077e4 f   lmathlib.obj
 0001:0000680b       _math_log10@4              1000780b f   lmathlib.obj
 0001:00006832       _math_exp@4                10007832 f   lmathlib.obj
 0001:00006859       _math_deg@4                10007859 f   lmathlib.obj
 0001:0000688e       _math_rad@4                1000788e f   lmathlib.obj
 0001:000068c3       _math_frexp@4              100078c3 f   lmathlib.obj
 0001:0000690b       _math_ldexp@4              1000790b f   lmathlib.obj
 0001:00006945       _math_min@4                10007945 f   lmathlib.obj
 0001:000069b4       _math_max@4                100079b4 f   lmathlib.obj
 0001:00006a25       _math_random@4             10007a25 f   lmathlib.obj
 0001:00006b42       _math_randomseed@4         10007b42 f   lmathlib.obj
 0001:00006baf       _math_pow@4                10007baf f   lmathlib.obj
 0001:00006e67       _adjust_mult_assign@12     10007e67 f   lparser.obj
 0001:00006eaf       _adjustlocalvars@8         10007eaf f   lparser.obj
 0001:00006ee6       _assignment@12             10007ee6 f   lparser.obj
 0001:00006f86       _block@4                   10007f86 f   lparser.obj
 0001:00006fba       _block_follow@4            10007fba f   lparser.obj
 0001:00006fe4       _body@12                   10007fe4 f   lparser.obj
 0001:0000706c       _breakstat@4               1000806c f   lparser.obj
 0001:000070c3       _check@8                   100080c3 f   lparser.obj
 0001:000070e2       _check_condition@12        100080e2 f   lparser.obj
 0001:000070f9       _check_match@16            100080f9 f   lparser.obj
 0001:0000716d       _checkname@4               1000816d f   lparser.obj
 0001:00007185       _chunk@4                   10008185 f   lparser.obj
 0001:000071b0       _close_func@4              100081b0 f   lparser.obj
 0001:00007271       _code_params@12            10008271 f   lparser.obj
 0001:000072d3       _code_string@8             100082d3 f   lparser.obj
 0001:000072ef       _cond@8                    100082ef f   lparser.obj
 0001:00007312       _constructor@4             10008312 f   lparser.obj
 0001:000073b6       _constructor_part@8        100083b6 f   lparser.obj
 0001:0000741e       _enterbreak@8              1000841e f   lparser.obj
 0001:0000743c       _error_expected@8          1000843c f   lparser.obj
 0001:00007474       _exp1@4                    10008474 f   lparser.obj
 0001:0000749a       _explist1@4                1000849a f   lparser.obj
 0001:000074ec       _expr@8                    100084ec f   lparser.obj
 0001:000074fe       _forbody@16                100084fe f   lparser.obj
 0001:0000756d       _forlist@8                 1000856d f   lparser.obj
 0001:000075e8       _fornum@8                  100085e8 f   lparser.obj
 0001:00007662       _forstat@8                 10008662 f   lparser.obj
 0001:000076df       _funcargs@8                100086df f   lparser.obj
 0001:0000776e       _funcname@8                1000876e f   lparser.obj
 0001:000077c8       _funcstat@8                100087c8 f   lparser.obj
 0001:00007841       _getbinopr@4               10008841 f   lparser.obj
 0001:000078c6       _getunopr@4                100088c6 f   lparser.obj
 0001:000078de       _ifstat@8                  100088de f   lparser.obj
 0001:000079a1       _indexupvalue@8            100089a1 f   lparser.obj
 0001:00007a12       _leavebreak@8              10008a12 f   lparser.obj
 0001:00007a36       _listfields@4              10008a36 f   lparser.obj
 0001:00007ab8       _localstat@4               10008ab8 f   lparser.obj
 0001:00007b07       _lookahead@4               10008b07 f   lparser.obj
 0001:00007b1d       _luaI_registerlocalvar@8   10008b1d f   lparser.obj
 0001:00007bd3       _namestat@4                10008bd3 f   lparser.obj
 0001:00007c29       _new_localvar@12           10008c29 f   lparser.obj
 0001:00007c9e       _new_localvarstr@12        10008c9e f   lparser.obj
 0001:00007cbe       _next@4                    10008cbe f   lparser.obj
 0001:00007cf5       _open_func@8               10008cf5 f   lparser.obj
 0001:00007d4f       _optional@8                10008d4f f   lparser.obj
 0001:00007d6c       _parlist@4                 10008d6c f   lparser.obj
 0001:00007e16       _pushclosure@8             10008e16 f   lparser.obj
 0001:00007ea7       _pushupvalue@8             10008ea7 f   lparser.obj
 0001:00007f70       _recfield@4                10008f70 f   lparser.obj
 0001:00007fc6       _recfields@4               10008fc6 f   lparser.obj
 0001:00008027       _removelocalvars@8         10009027 f   lparser.obj
 0001:0000805f       _repeatstat@8              1000905f f   lparser.obj
 0001:000080d1       _retstat@4                 100090d1 f   lparser.obj
 0001:0000810f       _search_local@12           1000910f f   lparser.obj
 0001:00008170       _simpleexp@8               10009170 f   lparser.obj
 0001:00008260       _singlevar@12              10009260 f   lparser.obj
 0001:000082a4       _stat@4                    100092a4 f   lparser.obj
 0001:000083a4       _str_checkname@4           100093a4 f   lparser.obj
 0001:000083ce       _string_constant@8         100093ce f   lparser.obj
 0001:0000841f       _subexpr@12                1000941f f   lparser.obj
 0001:000084c9       _test_then_block@8         100094c9 f   lparser.obj
 0001:000084f8       _var_or_func@8             100094f8 f   lparser.obj
 0001:00008549       _var_or_func_tail@8        10009549 f   lparser.obj
 0001:00008618       _whilestat@8               10009618 f   lparser.obj
 0001:000086c2       _errormessage@4            100096c2 f   lstate.obj
 0001:000086f5       _f_luaopen@8               100096f5 f   lstate.obj
 0001:00008870       _hash_s@8                  10009870 f   lstring.obj
 0001:00008b72       _newentry@16               10009b72 f   lstring.obj
 0001:00008bb0       _str_find@4                10009bb0 f   lstrlib.obj
 0001:00008d4f       _str_gsub@4                10009d4f f   lstrlib.obj
 0001:00008eea       _str_format@4              10009eea f   lstrlib.obj
 0001:00009128       _str_len@4                 1000a128 f   lstrlib.obj
 0001:00009167       _str_sub@4                 1000a167 f   lstrlib.obj
 0001:0000920e       _str_lower@4               1000a20e f   lstrlib.obj
 0001:00009294       _str_upper@4               1000a294 f   lstrlib.obj
 0001:0000931a       _str_rep@4                 1000a31a f   lstrlib.obj
 0001:00009382       _str_byte@4                1000a382 f   lstrlib.obj
 0001:00009403       _str_char@4                1000a403 f   lstrlib.obj
 0001:0000949a       _add_s@12                  1000a49a f   lstrlib.obj
 0001:00009579       _capture_to_close@8        1000a579 f   lstrlib.obj
 0001:000095a7       _check_capture@12          1000a5a7 f   lstrlib.obj
 0001:000095d5       _end_capture@16            1000a5d5 f   lstrlib.obj
 0001:0000962e       _lmemfind@16               1000a62e f   lstrlib.obj
 0001:00009699       _luaI_addquoted@12         1000a699 f   lstrlib.obj
 0001:000097f3       _match@16                  1000a7f3 f   lstrlib.obj
 0001:000099b4       _match_capture@16          1000a9b4 f   lstrlib.obj
 0001:000099f8       _match_class@8             1000a9f8 f   lstrlib.obj
 0001:00009b78       _matchbalance@16           1000ab78 f   lstrlib.obj
 0001:00009bd9       _matchbracketclass@12      1000abd9 f   lstrlib.obj
 0001:00009c56       _max_expand@20             1000ac56 f   lstrlib.obj
 0001:00009cb4       _min_expand@20             1000acb4 f   lstrlib.obj
 0001:00009cfb       _posrelat@8                1000acfb f   lstrlib.obj
 0001:00009d0e       _push_captures@8           1000ad0e f   lstrlib.obj
 0001:00009d66       _start_capture@16          1000ad66 f   lstrlib.obj
 0001:00009e23       _luaH_getany@12            1000ae23 f   ltable.obj
 0001:0000a198       _numuse@4                  1000b198 f   ltable.obj
 0001:0000a1b9       _rehash@8                  1000b1b9 f   ltable.obj
 0001:0000a275       _setnodevector@12          1000b275 f   ltable.obj
 0001:0000a2ef       _checktag@8                1000b2ef f   ltm.obj
 0001:0000a312       _findevent@4               1000b312 f   ltm.obj
 0001:0000a34b       _init_entry@8              1000b34b f   ltm.obj
 0001:0000a376       _luaI_checkevent@12        1000b376 f   ltm.obj
 0001:0000a62d       _LoadBlock@20              1000b62d f   lundump.obj
 0001:0000a682       _LoadChunk@8               1000b682 f   lundump.obj
 0001:0000a6a0       _LoadCode@16               1000b6a0 f   lundump.obj
 0001:0000a717       _LoadConstants@16          1000b717 f   lundump.obj
 0001:0000a7ed       _LoadFunction@12           1000b7ed f   lundump.obj
 0001:0000a898       _LoadHeader@8              1000b898 f   lundump.obj
 0001:0000aa30       _LoadInt@12                1000ba30 f   lundump.obj
 0001:0000aa4e       _LoadLines@16              1000ba4e f   lundump.obj
 0001:0000aa94       _LoadLocals@16             1000ba94 f   lundump.obj
 0001:0000ab14       _LoadNumber@12             1000bb14 f   lundump.obj
 0001:0000ab34       _LoadSignature@8           1000bb34 f   lundump.obj
 0001:0000ab7e       _LoadSize@12               1000bb7e f   lundump.obj
 0001:0000ab9c       _LoadString@12             1000bb9c f   lundump.obj
 0001:0000abf7       _LoadVector@24             1000bbf7 f   lundump.obj
 0001:0000ac80       _TestSize@16               1000bc80 f   lundump.obj
 0001:0000acbe       _ZNAME@4                   1000bcbe f   lundump.obj
 0001:0000acd1       _ezgetc@8                  1000bcd1 f   lundump.obj
 0001:0000ad0a       _ezread@16                 1000bd0a f   lundump.obj
 0001:0000adba       _unexpectedEOZ@8           1000bdba f   lundump.obj
 0001:0000addf       _adjust_varargs@12         1000bddf f   lvm.obj
 0001:0000ae13       _call_arith@12             1000be13 f   lvm.obj
 0001:0000ae42       _call_binTM@12             1000be42 f   lvm.obj
 0001:0000aeef       _luaV_closure@8            1000beef f   lvm.obj
 0001:0000b8ca       $LN178                     1000c8ca     lvm.obj
 0001:0000bb6b       _luaV_pack@8               1000cb6b f   lvm.obj
 0001:0000bdbb       _luaV_strcomp@8            1000cdbb f   lvm.obj
 0001:0000c000       _traceexec@16              1000d000 f   lvm.obj
 0001:0000c141       _zffilbuf@4                1000d141 f   lzio.obj
 0001:0000c190       _zmfilbuf@4                1000d190 f   lzio.obj
 0001:0000c196       ?alloc@@YGPAXI@Z           1000d196 f   LuaMem.obj
 0001:0000c57e       __catch$?_Copy@?$basic_string@DU?$char_traits@D@std@@V?$allocator@D@2@@std@@QAEXII@Z$0 1000d57e f i Assist:pch.obj
 0001:0000c604       __catch$?_Copy@?$basic_string@DU?$char_traits@D@std@@V?$allocator@D@2@@std@@QAEXII@Z$1 1000d604 f i Assist:pch.obj
 0001:0000cb50       $$000000                   1000db50     MSVCRT:ftol2.obj
 0001:0000ce4e       _pre_c_init                1000de4e f   MSVCRT:crtdll.obj
 0001:0000d0b9       ___DllMainCRTStartup       1000e0b9 f   MSVCRT:crtdll.obj
 0001:0000d224       $$000000                   1000e224     MSVCRT:ehprolog.obj
 0001:0000d400       $$000000                   1000e400     MSVCRT:sehprolg4.obj
 0001:0000d761       ?ArrayUnwindFilter@@YAHPAU_EXCEPTION_POINTERS@@@Z 1000e761 f   MSVCRT:ehvecdtr.obj
 0001:0000db6c       __ehhandler$?_Copy@?$basic_string@DU?$char_traits@D@std@@V?$allocator@D@2@@std@@QAEXII@Z 1000eb6c f   Assist:pch.obj
 0001:0000db76       ??__Es_pool@@YAXXZ         1000eb76 f   LuaMem.obj
 0001:0000db94       ??__E?_Generic_object@?$_Error_objects@H@std@@2V_Generic_error_category@2@A@@YAXXZ 1000eb94 f   Assist:pch.obj
 0001:0000dba0       ??__E?_Iostream_object@?$_Error_objects@H@std@@2V_Iostream_error_category@2@A@@YAXXZ 1000eba0 f   Assist:pch.obj
 0001:0000dbac       ??__E?_System_object@?$_Error_objects@H@std@@2V_System_error_category@2@A@@YAXXZ 1000ebac f   Assist:pch.obj
 0001:0000dbb8       ??__E?id@?$num_put@DV?$back_insert_iterator@V?$basic_string@DU?$char_traits@D@std@@V?$allocator@D@2@@std@@@std@@@std@@2V0locale@2@A@@YAXXZ 1000ebb8 f   Assist:pch.obj
 0001:0000dbc6       ??__E?id@?$num_put@_WV?$back_insert_iterator@V?$basic_string@_WU?$char_traits@_W@std@@V?$allocator@_W@2@@std@@@std@@@std@@2V0locale@2@A@@YAXXZ 1000ebc6 f   Assist:pch.obj
 0001:0000dbd4       ??__Fs_pool@@YAXXZ         1000ebd4 f   LuaMem.obj
 0001:0000dbdf       ??__F?_Generic_object@?$_Error_objects@H@std@@2V_Generic_error_category@2@A@@YAXXZ 1000ebdf f   Assist:pch.obj
 0001:0000dbea       ??__F?_Iostream_object@?$_Error_objects@H@std@@2V_Iostream_error_category@2@A@@YAXXZ 1000ebea f   Assist:pch.obj
 0001:0000dbf5       ??__F?_System_object@?$_Error_objects@H@std@@2V_System_error_category@2@A@@YAXXZ 1000ebf5 f   Assist:pch.obj
 0002:000001e4       _s_pool$initializer$       1000f1e4     LuaMem.obj
 0002:000001e8       ?_Generic_object$initializer$@?$_Error_objects@H@std@@2P6AXXZA 1000f1e8     Assist:pch.obj
 0002:000001ec       ?_Iostream_object$initializer$@?$_Error_objects@H@std@@2P6AXXZA 1000f1ec     Assist:pch.obj
 0002:000001f0       ?_System_object$initializer$@?$_Error_objects@H@std@@2P6AXXZA 1000f1f0     Assist:pch.obj
 0002:000001f4       ?id$initializer$@?$num_put@DV?$back_insert_iterator@V?$basic_string@DU?$char_traits@D@std@@V?$allocator@D@2@@std@@@std@@@std@@2P6AXXZA 1000f1f4     Assist:pch.obj
 0002:000001f8       ?id$initializer$@?$num_put@_WV?$back_insert_iterator@V?$basic_string@_WU?$char_traits@_W@std@@V?$allocator@_W@2@@std@@@std@@@std@@2P6AXXZA 1000f1f8     Assist:pch.obj
 0002:00000204       _pcinit                    1000f204     MSVCRT:crtdll.obj
 0002:00000208       _pinit                     1000f208     MSVCRT:atonexit.obj
 0002:0000020c       _pinit                     1000f20c     MSVCRT:cpu_disp.obj
 0002:00000538       ?errornames@?1??passresults@@9@9 1000f538     lbaselib.obj
 0002:00000550       _deprecated_names          1000f550     lbaselib.obj
 0002:00000570       _min_funcs                 1000f570     lbaselib.obj
 0002:00000590       _base_funcs                1000f590     lbaselib.obj
 0002:00000a40       _codes                     1000fa40     lcode.obj
 0002:00000bc0       _dblib                     1000fbc0     ldblib.obj
 0002:00000e28       ?mode@?1??io_seek@@9@9     1000fe28     liolib.obj
 0002:00000e34       ?modenames@?1??io_seek@@9@9 1000fe34     liolib.obj
 0002:00000e44       _miniolib                  1000fe44     liolib.obj
 0002:00000e50       _iolib                     1000fe50     liolib.obj
 0002:00000e98       _iolibtag                  1000fe98     liolib.obj
 0002:00000ee0       _filenames                 1000fee0     liolib.obj
 0002:00001180       _token2string              10010180     llex.obj
 0002:000013c0       _mathlib                   100103c0     lmathlib.obj
 0002:00001660       _priority                  10010660     lparser.obj
 0002:00001910       _strlib                    10010910     lstrlib.obj
 0002:00001bd0       _luaT_validevents          10010bd0     ltm.obj
 0002:00002338       _GS_ExceptionPointers      10011338     MSVCRT:gs_report.obj
 0002:00002588       __catchsym$?_Copy@?$basic_string@DU?$char_traits@D@std@@V?$allocator@D@2@@std@@QAEXII@Z$5 10011588     Assist:pch.obj
 0002:00002598       __catchsym$?_Copy@?$basic_string@DU?$char_traits@D@std@@V?$allocator@D@2@@std@@QAEXII@Z$4 10011598     Assist:pch.obj
 0002:000025a8       __unwindtable$?_Copy@?$basic_string@DU?$char_traits@D@std@@V?$allocator@D@2@@std@@QAEXII@Z 100115a8     Assist:pch.obj
 0002:000025c8       __ehfuncinfo$?_Copy@?$basic_string@DU?$char_traits@D@std@@V?$allocator@D@2@@std@@QAEXII@Z 100115c8     Assist:pch.obj
 0002:000025ec       __tryblocktable$?_Copy@?$basic_string@DU?$char_traits@D@std@@V?$allocator@D@2@@std@@QAEXII@Z 100115ec     Assist:pch.obj
 0002:00002618       __sehtable$__onexit        10011618     MSVCRT:atonexit.obj
 0002:00002638       __sehtable$___DllMainCRTStartup 10011638     MSVCRT:crtdll.obj
 0002:00002660       __sehtable$__IsNonwritableInCurrentImage 10011660     MSVCRT:pesect.obj
 0002:00002680       __sehtable$??_M@YGXPAXIHP6EX0@Z@Z 10011680     MSVCRT:ehvecdtr.obj
 0002:000026a0       __sehtable$?__ArrayUnwind@@YGXPAXIHP6EX0@Z@Z 100116a0     MSVCRT:ehvecdtr.obj
 0002:0000295a       .idata$6                   1001195a     Debug:Debug.dll
 0002:000029f0       .idata$6                   100119f0     Memory:Memory.dll
 0002:00002ab2       .idata$6                   10011ab2     msvcprt:MSVCP110.dll
 0002:00002d9e       .idata$6                   10011d9e     MSVCRT:MSVCR110.dll
 0002:00002fb2       .idata$6                   10011fb2     kernel32:KERNEL32.dll
 0002:00002fc0       .edata                     10011fc0     lua.exp
 0002:00002fe8       rgpv                       10011fe8     lua.exp
 0002:00003160       rgszName                   10012160     lua.exp
 0002:000032d8       rgwOrd                     100122d8     lua.exp
 0002:00003394       szName                     10012394     lua.exp
 0002:0000339c       $N00001                    1001239c     lua.exp
 0002:000033a7       $N00002                    100123a7     lua.exp
 0002:000033bb       $N00003                    100123bb     lua.exp
 0002:000033cd       $N00004                    100123cd     lua.exp
 0002:000033de       $N00005                    100123de     lua.exp
 0002:000033f0       $N00006                    100123f0     lua.exp
 0002:00003401       $N00007                    10012401     lua.exp
 0002:00003415       $N00008                    10012415     lua.exp
 0002:0000342a       $N00009                    1001242a     lua.exp
 0002:0000343b       $N00010                    1001243b     lua.exp
 0002:0000344f       $N00011                    1001244f     lua.exp
 0002:00003462       $N00012                    10012462     lua.exp
 0002:00003475       $N00013                    10012475     lua.exp
 0002:00003486       $N00014                    10012486     lua.exp
 0002:00003498       $N00015                    10012498     lua.exp
 0002:000034ac       $N00016                    100124ac     lua.exp
 0002:000034bf       $N00017                    100124bf     lua.exp
 0002:000034d2       $N00018                    100124d2     lua.exp
 0002:000034de       $N00019                    100124de     lua.exp
 0002:000034f1       $N00020                    100124f1     lua.exp
 0002:000034fe       $N00021                    100124fe     lua.exp
 0002:0000350b       $N00022                    1001250b     lua.exp
 0002:00003519       $N00023                    10012519     lua.exp
 0002:00003530       $N00024                    10012530     lua.exp
 0002:00003541       $N00025                    10012541     lua.exp
 0002:00003552       $N00026                    10012552     lua.exp
 0002:00003560       $N00027                    10012560     lua.exp
 0002:00003570       $N00028                    10012570     lua.exp
 0002:0000357e       $N00029                    1001257e     lua.exp
 0002:0000358b       $N00030                    1001258b     lua.exp
 0002:0000359d       $N00031                    1001259d     lua.exp
 0002:000035b3       $N00032                    100125b3     lua.exp
 0002:000035c4       $N00033                    100125c4     lua.exp
 0002:000035d6       $N00034                    100125d6     lua.exp
 0002:000035e6       $N00035                    100125e6     lua.exp
 0002:000035f7       $N00036                    100125f7     lua.exp
 0002:00003603       $N00037                    10012603     lua.exp
 0002:00003611       $N00038                    10012611     lua.exp
 0002:00003622       $N00039                    10012622     lua.exp
 0002:00003632       $N00040                    10012632     lua.exp
 0002:00003647       $N00041                    10012647     lua.exp
 0002:00003655       $N00042                    10012655     lua.exp
 0002:00003663       $N00043                    10012663     lua.exp
 0002:00003674       $N00044                    10012674     lua.exp
 0002:00003687       $N00045                    10012687     lua.exp
 0002:00003697       $N00046                    10012697     lua.exp
 0002:000036a7       $N00047                    100126a7     lua.exp
 0002:000036b8       $N00048                    100126b8     lua.exp
 0002:000036cb       $N00049                    100126cb     lua.exp
 0002:000036e1       $N00050                    100126e1     lua.exp
 0002:000036f5       $N00051                    100126f5     lua.exp
 0002:00003705       $N00052                    10012705     lua.exp
 0002:00003713       $N00053                    10012713     lua.exp
 0002:00003726       $N00054                    10012726     lua.exp
 0002:00003732       $N00055                    10012732     lua.exp
 0002:0000373e       $N00056                    1001273e     lua.exp
 0002:0000374b       $N00057                    1001274b     lua.exp
 0002:00003760       $N00058                    10012760     lua.exp
 0002:00003774       $N00059                    10012774     lua.exp
 0002:00003783       $N00060                    10012783     lua.exp
 0002:00003796       $N00061                    10012796     lua.exp
 0002:000037a8       $N00062                    100127a8     lua.exp
 0002:000037bc       $N00063                    100127bc     lua.exp
 0002:000037cd       $N00064                    100127cd     lua.exp
 0002:000037dd       $N00065                    100127dd     lua.exp
 0002:000037eb       $N00066                    100127eb     lua.exp
 0002:000037fb       $N00067                    100127fb     lua.exp
 0002:00003809       $N00068                    10012809     lua.exp
 0002:00003819       $N00069                    10012819     lua.exp
 0002:00003824       $N00070                    10012824     lua.exp
 0002:00003832       $N00071                    10012832     lua.exp
 0002:00003845       $N00072                    10012845     lua.exp
 0002:0000385b       $N00073                    1001285b     lua.exp
 0002:0000386c       $N00074                    1001286c     lua.exp
 0002:0000387e       $N00075                    1001287e     lua.exp
 0002:00003891       $N00076                    10012891     lua.exp
 0002:000038a2       $N00077                    100128a2     lua.exp
 0002:000038b2       $N00078                    100128b2     lua.exp
 0002:000038c0       $N00079                    100128c0     lua.exp
 0002:000038d5       $N00080                    100128d5     lua.exp
 0002:000038e3       $N00081                    100128e3     lua.exp
 0002:000038f5       $N00082                    100128f5     lua.exp
 0002:00003903       $N00083                    10012903     lua.exp
 0002:00003915       $N00084                    10012915     lua.exp
 0002:00003920       $N00085                    10012920     lua.exp
 0002:00003933       $N00086                    10012933     lua.exp
 0002:00003943       $N00087                    10012943     lua.exp
 0002:00003954       $N00088                    10012954     lua.exp
 0002:00003964       $N00089                    10012964     lua.exp
 0002:00003976       $N00090                    10012976     lua.exp
 0002:00003982       $N00091                    10012982     lua.exp
 0002:00003992       $N00092                    10012992     lua.exp
 0002:0000399f       $N00093                    1001299f     lua.exp
 0002:000039b3       $N00094                    100129b3     lua.exp
 0003:00000104       __Tuple_alloc              10013104     pch.obj
 0003:00000105       _ignore                    10013105     pch.obj
 0003:00000106       _allocator_arg             10013106     pch.obj
 0003:00000107       _piecewise_construct       10013107     pch.obj
 0003:00000110       _key1                      10013110     ldblib.obj
 0003:00000111       _key2                      10013111     ldblib.obj
 0003:00000114       _s_pool                    10013114     LuaMem.obj
 0003:00000124       __Tuple_alloc              10013124     Assist:pch.obj
 0003:00000125       _ignore                    10013125     Assist:pch.obj
 0003:00000126       _allocator_arg             10013126     Assist:pch.obj
 0003:00000127       _piecewise_construct       10013127     Assist:pch.obj
 0003:00000130       ___proc_attached           10013130     MSVCRT:crtdll.obj
 0003:00000148       _GS_ExceptionRecord        10013148     MSVCRT:gs_report.obj
 0003:00000198       _GS_ContextRecord          10013198     MSVCRT:gs_report.obj
 0003:00000464       _DebuggerWasPresent        10013464     MSVCRT:gs_report.obj
 0004:00000060       $R000000                   10014060     * linker generated manifest res *
